:020000040000fa
:08000000c01404000000000020
:020000040000fa
:1000080004140000081400000c1400001014000070
:1000180014140000bc140000bc140000bc14000040
:10002800181400001c140000201400002414000000
:10003800bc140000281400002c1400003014000028
:1000480034140000381400003c1400004014000070
:100058004414000048140000bc140000bc14000044
:100068004c140000501400005414000058140000f0
:100078005c140000bc140000bc140000bc14000098
:10008800bc14000060140000641400006814000030
:100098006c14000070140000741400007814000040
:1000a8007c14000080140000bc140000bc14000084
:1000b800bc14000084140000881400008c14000094
:1000c800bc14000090140000bc140000bc14000014
:1000d800bc14000094140000bc140000bc14000000
:1000e800bc140000981400009c140000bc1400000c
:1000f800bc140000bc140000bc140000bc140000b8
:10010800bc140000bc140000bc140000bc140000a7
:10011800bc140000bc140000a0140000bc140000b3
:10012800bc140000a4140000a8140000ac140000c3
:10013800bc140000bc140000bc140000bc14000077
:10014800b0140000bc140000bc140000bc14000073
:10015800bc140000b4140000bc140000bc1400005f
:10016800bc140000bc140000bc140000bc14000047
:10017800bc140000bc140000b8140000bc1400003b
:10018800bc140000bc140000bc140000bc14000027
:10019800bc140000bc140000bc140000bc14000017
:1001a800bc140000bc140000bc140000bc14000007
:1001b800bc140000bc140000bc140000bc140000f7
:1001c800bc140000bc140000bc140000bc140000e7
:1001d800bc140000bc140000bc140000bc140000d7
:1001e800bc140000bc140000bc140000bc140000c7
:0801f800bc140000bc1400005f
:020000040000fa
:10280000c014040000000000ea59040000000000a9
:10281000ea59040000000000ea590400000000002a
:10282000ea59040000000000ea590400000000001a
:10283000ea59040000000000ea590400000000000a
:10284000ea59040000000000ea59040000000000fa
:10285000ea59040000000000ea59040000000000ea
:10286000ea590400000000009c570400000000002a
:10287000ea59040000000000ea59040000000000ca
:10288000ea59040000000000ea59040000000000ba
:10289000ea59040000000000ea59040000000000aa
:1028a000ea59040000000000ea590400000000009a
:1028b000c03b040000000000ea59040000000000d2
:1028c000ea59040000000000ea590400000000007a
:1028d000ea59040000000000ea590400000000006a
:1028e000ea59040000000000ea590400000000005a
:1028f000ea59040000000000ea590400000000004a
:10290000ea59040000000000ea5904000000000039
:10291000ea59040000000000ea5904000000000029
:10292000ea59040000000000ea5904000000000019
:10293000ea59040000000000ea5904000000000009
:10294000ea59040000000000ea59040000000000f9
:10295000ea59040000000000ea59040000000000e9
:10296000ea59040000000000ea59040000000000d9
:102970009059040000000000ea5904000000000023
:020000040000fa
:10298000cf6421000e7f22000e01880000000000ad
:1029900000012000200288000c0007002080250094
:1029a0000100200011000700000020000000e000ee
:1029b0000200320000000200000000001455020076
:1029c000000000000040da000000fe004440a900c2
:1029d000c00520000000e0000300320000002000dd
:1029e000a00188004440a800000006009101880072
:1029f000800078000000eb0015003700e280400006
:102a000032a0b4009101ba00e280400032a0b400cc
:102a10009102ba00e280400032a0b4000002eb0054
:102a2000472bde00f507b200602ce10004003a00fd
:102a30000059eb008301e900fdff3e000400370070
:102a40006128e100010032000082eb000400070071
:102a50001101ba000200e000e8ff3a0000000600a1
:102a60003159ba008301e9000c0032002159ba0043
:102a70008301e900080032000400e00003003a008e
:102a8000e280400032a0b400f5ff370011d9ba004f
:102a90008301e900faff3a008100e800e18040008c
:102aa00032a0b4000000060000000000000000009a
:102ab0000000000000000000000000000000000016
:102ac0000000fa0016a2a9001682a8000080fa00f1
:102ad000000006000000fa0000000000b4108000b2
:102ae00061026200e00f5200fcff3a00b410800067
:102af00062026200e00f5200f8ff3a00b41080005a
:102b000064026200e00f5200f4ff3a00b41080004b
:102b100068026200e00f5200f0ff3a00b41080003b
:102b200070026200e00f5200ecff3a00c510800016
:102b30000400240004826200e00f5200e7ff3a0024
:102b40000080fa00000006000000fa001662a800eb
:102b500000000000b410800068026200e00f520024
:102b6000fcff3a0018c2a9008410800004427800db
:102b7000044078000080fa00000006000200fa001d
:102b8000004f78009e4278000582fb009410880078
:102b9000c51080000408200004826200e00f52008b
:102ba0000200320000c2eb00010037000042eb00df
:102bb000044078000080fa00000006000000fa00df
:102bc00016a2a8001682a8000080fa0000000600e5
:102bd0000400fa00000f7800110798001e02900010
:102be000a41088001e027800b41088000080fa004b
:102bf000000006000000fa001602a8000080fa009b
:102c0000000006000000fa001642a8000080fa004a
:102c100000000600839f68000100e00002003d0004
:102c200060001000e08018000300e00002003d009a
:102c300060011100e0811900050007004f00e0006d
:102c400002003b0060001000e08018000000060059
:102c50006022b800060220000000d0008180d2006f
:102c60000482d2008582d2000000a000020252003d
:102c700083825a00030031000202420083824a002c
:102c80000000a1000603e900f3ff3a00000006007f
:102c9000e4874700889fbe008a9fbe008c9fbe00cd
:102ca0008e1f780024a8200015548000e08f520069
:102cb0000b003a00e4024200155488006554880075
:102cc0002402980054548800a44290000504a000f7
:102cd00025429800e44290000504a0006542980057
:102ce000670440004244de004244dd00525480004c
:102cf00044a92000c96421008484540025002000d8
:102d0000110009008504d80080bf9f00050744001a
:102d10000e0747000003eb00e4054400fc642100bb
:102d20000406560008064600020037001600200080
:102d30000d01780022429000610262000200320020
:102d40000a003700150978009202780025429000a9
:102d500061026200fbff320008024100848f5200d2
:102d600002003900e00f54003f003d009206780059
:102d70000d00a100828f5600edff3e00e10f5300d1
:102d8000eaff3a000fba9700840f540002003600a1
:102d9000890f5400100039006143b800614ab9003e
:102da000b0ff2f000100200004025000858258006f
:102db000840f5300858f5b00020035000b057800ff
:102dc00006003700110009000986d8000982b90001
:102dd00004057800010037000e0578000a0078002d
:102de00089000700e10f400005003a000b0578005c
:102df0000b00780084000700e10f40002b00320038
:102e000064548000000a7800645480006403420027
:102e1000a4429000860f5000020032000504a0007a
:102e2000010037000504a100254298006405550003
:102e30000a0540000a0878006a54880024a8200087
:102e4000040d780065548000254290000404a00021
:102e5000a4429800204290000404a100244098005d
:102e60000003eb00b2ff370054548800848f5200f7
:102e7000070036001403be0076548800875488008b
:102e8000120a78008042eb005454800025429800da
:102e90005754800007097800224290000404a000e3
:102ea0002441980064004100010037000000eb005d
:102eb0004f0778004f06be004f05be004f04be000e
:102ec0004f00b10000000600e00f50000800320083
:102ed0006400500054548000840f50000100310001
:102ee00050548800204290000404a100244098001f
:102ef00000000600889fbe008a9fbe000004be003e
:102f0000e08f540005003a00e00f54003200320018
:102f100008007800ecff070030003700e00f540095
:102f200004003a000900780059ff07008004780087
:102f30002a003700640254009405780068fa97006c
:102f4000610262000200320008007800deff070024
:102f5000090078004eff070080047800e08f5400dd
:102f60001e003200888f54001b00320069bd97009c
:102f70000905550042d5de0088855500c2ddde001a
:102f80000a0178008b0f5500010036000b01780014
:102f90004211dd0088007800090078001300070066
:102fa000888f54000d0031004255dd000a85440031
:102fb000880f5500090036000804550042c4de00a1
:102fc0004244dd000884440074548000855480002d
:102fd000048cbe00010037008804780009007800e6
:102fe0004f05be004f04be0000000600000278003e
:102ff00002003700315a78000201e900e00f510069
:10300000fcff3a0000000600889fbe0080047800a4
:1030100090548000e00f500004003a000e000700ba
:103020000084eb00e00f5000080035009854800049
:10303000e08f54000500320009004400060007003c
:10304000e00f500001003d000084eb000800780014
:103050004f04be0000000600e00f500004003a00dc
:1030600044a920009454880000027800060037002c
:103070000082eb00c5642100850f500002003e0075
:10308000905488000002eb00040078000000060065
:020000040000fa
:103090000d0a000052790000732000005553000013
:1030a00042200000666f000072200000416d0000a9
:1030b0006967000061200000436f00006d70000030
:1030c0007574000065720000730d00000a2800008e
:1030d0006329000032300000323100002d32000040
:1030e0003032000036200000372d000062690000f9
:1030f000742c000020410000727400007572000002
:10310000204700006164000061770000736b0000dd
:10311000690d00000a760000302e000031360000f4
:103120000d0a0000000000003031000032330000c2
:1031300034350000363700003839000041420000c5
:08314000434400004546000075
:020000040000fa
:10314800705180004600de0061406000000006000b
:1031580004f02000a65080008602620010c3b3006d
:10316800e08f52001e003200a55080000503620067
:1031780005402000850f530007003a00a450800046
:10318800040fb2000040e900f00f520014003a00aa
:103198006a40400000000600a65080000602620057
:1031a80005502000850f520002003a0022cabf00d5
:1031b80000000600a550800040c3b30004102000a2
:1031c800848f520006003600a550800000c0e90038
:1031d800f43f2000848f52000100360000c0e80050
:1031e800000006008042780060c0b30014a22000ee
:1031f8001442780084cf520008003a0004f02000fe
:10320800a55080000502620030c0b300e00f5200f4
:1032180002003200142aef000040eb000000060014
:103228008042780060c0b30014a2200014427800e5
:1032380084cf520007003a00a550800030c0b30088
:1032480004412000848f520002003a00142aec0046
:103258000040eb00000006008042780060c0b30028
:1032680014a220001442780084cf520009003a00ca
:10327800a550800030c0b30004402000848f520065
:1032880004003a009404a90070024200a450880087
:103298000040eb0000000600b4508000940290004b
:1032a8000560a10015029800940290000550a10045
:1032b80015029800684aed0068eab700030032007a
:1032c80000ff2f00142ab60000000600694aed002e
:1032d80069eab7000411200003003a0070c0b30087
:1032e80022eab70004502000a4508800000006001d
:1032f8000a00fa00889fbe008a9fbe008c9fbe000d
:10330800804478000144780082467800dc538000cd
:103318002b0020000005eb004352dd00660342004d
:10332800459e200065037b008603d100e1c363004e
:10333800e1cf53003b003a004533de0061436300b0
:1033480003003a00e5427a0089cf520035003a007e
:1033580066034200459e200065037b004433de007f
:103368006143630004003a00048242001442900062
:10337800884f52002b003a00c352dd00668342009a
:10338800449e200064037b004333de0061436300f6
:1033980004003a008582e80064c27a008d4f52002a
:1033a80020003a000c4a90000482fb009c4a9000de
:1033b800c82add0084827200d5b79f00ac4a90000d
:1033c8008582fb003c4a90004822dd00050272001d
:1033d800e4b79f00e9ef9f00f8ef9f008df79f008b
:1033e8008400200005002000768157009107200006
:1033f80000c0eb0093bf9f00ef1c07009fb9970028
:10340800e04f500007003a004355dd00849e20003d
:10341800040545001a4590008a49780010c0b30099
:10342800040037000a05e8008b05e900baff3a00f6
:103438000b4078004f06be004f05be004f04be008b
:103448000080fa00000006000800fa00889fbe000d
:103458008a9fbe00d95380002ecaa9002eeaa9006f
:103468002b0020000005eb00489e20004352dd00a1
:10347800e6024200e8827a000503d1006143630056
:103488000f00320068437a00c9429000854f53000c
:103498004f003a008402440015439000d94290003e
:1034a800854f53004a003a000482e800e8427a0057
:1034b8006942900084cf520045003a00430037002b
:1034c800894b90008783fb00194b90004833dd003f
:1034d80007037300e8037a00868f530019003a0047
:1034e8008483e800294890000080fb00394b900055
:1034f8004833dd0000037300e8837b00868f5300a8
:1035080010003a00472bde0061436300e14f53008f
:103518000b003a002eeaa8006402420004034400ab
:103528001640900024eab700c22ade00e1c2620019
:103538000400320068407a001eeab7000100370034
:103548002ecaa8004352dd00e8027a00e18f42004b
:103558001f003a008482e80068807a00e10f40008a
:103568001b003a00094b90000683fb00994b900022
:10357800c83bdd008683730087bf9f00a94b90007e
:103588008783fb00394b90004833dd000703730045
:1035980096bf9f0068437a00c6f79f000402440064
:1035a80014429000d4f79f00e8c27a00e5f79f0024
:1035b800840020000500200070815700910720003a
:1035c8007d1c0700e04f500001003a002ecaa800f9
:1035d8002ecaab000f0032004355dd00e40245005f
:1035e800449e2000050342001640900023eab700dd
:1035f8006605450064037d004233de0061436300d5
:103608001bc0b3000600320064c07a001eeab7008f
:10361800030037000a05e8008b05e90093ff3a002c
:103628000b4078004f05be004f04be000080fa0032
:103638000000060080427800e0cf520002003a0005
:103648006051800000000600545180000c003700d3
:1036580024039000e00f5300080032002600900079
:1036680004003700205b9000854f530007003200ac
:1036780010007800e00f5000faff3a0014027800ba
:10368800e00f5200f2ff3a00040078000000060044
:103698000200fa00881f78000204780014a22000b3
:1036a80014427800844f50000500320064c0b30013
:1036b800044c78008009eb00b31178002200370031
:1036c80001407800e3bf9f00daff0700efb99700d9
:1036d800e00f50001a00320090029000c92ade0064
:1036e800e1c26200100290000410b200050032002e
:1036f800004ceb00000b9000900b90008689be00f8
:103708000d003700100290000402b20002003200df
:1037180014c1b30007003700100290000404b2007f
:103728000300320040589000004c78000200370037
:1037380094c1b300044c78000540780003003700ba
:1037480044c1b300044c780010c0b3004f047800a3
:103758000080fa000000060014a22000144278003d
:10376800844f50000a003a0001407800b1ff07007a
:10377800e00f500006003200100290000470a00014
:1037880014009800100290000490a0001400980003
:10379800000006000200fa00881f78000042780046
:1037a8000204780065c0b30016a220001643780012
:1037b800864f52000f003a0001407800e3bf9f0097
:1037c8009cff070045c1b300efb99700e00f500018
:1037d80008003200610464004d44dd0010029000ce
:1037e80004d0a10008027200140098000310980089
:1037f8008042eb00054078004f0478000080fa0012
:1038080000000600004278000140780065c0b3005f
:1038180016a2200016437800864f52000b003a008b
:1038280084ff070045c1b300e00f500007003200d5
:10383800100290000450a10014009800100290009b
:103848000460a100140098008042eb000540780055
:1038580000000600645180008083fb00d40a9000b9
:10386800c82ade00e3826200878f520003003a0014
:10387800940290000520b200210032001b6aef007c
:1038880055518000e08f520026003a00050278006a
:1038980028003700e00f52001f003200540b900040
:1038a8004833de0063036300870f530017003a00b4
:1038b800e04f500003003200e34f500013003a007d
:1038c80003003700140390000620b2000a003700f6
:1038d800140390000620b200060032003403900062
:1038e800e00f530009003a002403900036029800c4
:1038f8000600370034039000e00f530003003a003d
:10390800b450880015c0b3000c00370014027800ca
:10391800e00f520007003a0095027800e08f52004d
:103928000600320025029000e00f5200010032002c
:1039380024029000e08f5200d6ff3a00054078003c
:1039480000000600889fbe008a1f78001800370014
:10395800140478001000370094047800050037003c
:103968001005780056fd070054518000140290009d
:103978002a029800545180001402900024009000fc
:10398800e00f5000f6ff3a00040078004cfd0700f5
:103998005451800019029800505180001002900084
:1039a800e00f5200ecff3a0045fd0700585188002f
:1039b80054518000e00f5200e5ff3a002c0af8004d
:1039c800160af9004f0578004f04be0000000600f3
:1039d800889fbe0007003700980490001800780000
:1039e80037fd0700405180000008eb0034fd070058
:1039f8004951880048518000e00f5400f6ff3a0012
:103a0800d0538000e00f5000020032002cfd070068
:103a1800d853880080518000e00f50000200320027
:103a280027fd0700302aef00c6ff07004f04be003d
:103a380000000600881f780068518000e00f5400dd
:103a480007003a00200220008ffc07006051880020
:103a5800e00f50000f00320008087800010037001e
:103a6800dbff07002c0af800160af900142aef00f9
:103a780010aaef00206aef00216aef006a0aa80086
:103a88004400200094518800a4518800362aef0091
:103a980010c0b3004f0478000000060090029000a8
:103aa8000550a10015009800900290000560a10043
:103ab80015009800900290000570a100150098006c
:103ac800900290000580a100150098001003900056
:103ad80005fe2f00850263001500980090029000f3
:103ae80005c0a10015009800330898006033b8009d
:103af8000608980017089800050020005400980050
:103b0800650098000002eb007408980021089800ee
:103b18007200980004c2b300045898001002900084
:103b28000490a10014009800000006009002900084
:103b38000550a10015009800900290000560a100b2
:103b480015009800900290000570a10015009800db
:103b5800900290000580a1001500980010039000c5
:103b680005fe2f0085026300150098009002900062
:103b780005c0a10015009800330898006033b8000c
:103b880006089800170898006123b80056009800a6
:103b9800670098008002eb007508980021089800db
:103ba80072009800850f520002003a0004c1b30069
:103bb8000100370004c3b3000458980010029000b5
:103bc8000490a10014009800000006001002900064
:103bd8000470a10014009800100290000480a10055
:103be800140098009002900004fe2f0004826200e6
:103bf800140098001002900004c0a100140098005e
:103c0800310898006022b800040898001508980048
:103c18000300200052009800630098008002eb0027
:103c280075089800500a90000430b2000630200051
:103c3800860f520002003a0004c4b300080037009f
:103c480006102000860f520004003a0004c6b30094
:103c580004589800954098000200370004c8b30043
:103c680004589800100290000490a10014009800d5
:103c7800000006000400fa00889fbe000043780098
:103c8800020478000401be0064c0b30015a220003d
:103c980095427800854f530026003a0006f0200030
:103ca800a45080000403630014c0b3000540200042
:103cb800850f53001f003a0001407800c2bf9f00e3
:103cc800d3bf9f005bfe070044c1b3004fb9970004
:103cd800e00f500017003200d00a90000530b20003
:103ce80084c1b30013003200a05a900054c1b3003d
:103cf800e0cf52000f003d00900290000502b20094
:103d080014c1b3000b003a00900490000904b200fb
:103d180024c1b30007003a00900290000520b200c9
:103d280004c1b3000300320088007800a7ff070031
:103d380009427800044078004f04be000080fa0071
:103d480000000600100290000470a1001400980002
:103d5800100290000480a1001400980090029000c6
:103d680004fe2f00048262001400980010029000e4
:103d780004c0a10014009800310898006022b8001f
:103d880004089800150898000300200052009800c5
:103d9800630098008002eb0075089800500a9000b4
:103da8000430b20006302000860f520002003a00ac
:103db80004c5b3000800370006102000860f520023
:103dc80004003a0004c7b3000458980095409800ce
:103dd8000200370004c9b30004589800100290008c
:103de8000490a10014009800000006000400fa00e6
:103df800889fbe0000437800020478000401be00da
:103e080064c0b30015a2200095427800854f530086
:103e180026003a0006f02000a45080000403630046
:103e280014c0b30005402000850f53001f003a005e
:103e380001407800c2bf9f00d3bf9f00fdfd07006f
:103e480044c1b3004fb99700e00f5000170032008b
:103e5800d00a90000530b20084c1b30013003200cc
:103e6800a05a900054c1b300e0cf52000f003500b3
:103e7800900290000502b20014c1b3000b003a0092
:103e8800900490000904b20024c1b30007003a006e
:103e9800900290000520b20004c1b3000300320074
:103ea80088007800a7ff07000942780004407800de
:103eb8004f04be000080fa00000006000200fa006d
:103ec800889fbe008a9fbe008c9fbe000045780078
:103ed800010478008204780024072000840f54002d
:103ee80003003200f4ff2700840f540009003a0051
:103ef80019489000e14f400026003200a2c0b300ec
:103f08000440bc000280e800a49d200064037800ff
:103f18001b0037005b518000611eb8000e0037009f
:103f28007b409000a2c0b3000440bc000281e800be
:103f3800a49d2000640379000c02be0009017800ea
:103f4800880078000a40780093bf9f0006000100af
:103f58009b0578009fb99700e08f5500f0ff3a0065
:103f68002eeaab000b00320024cabf00a2c0b30087
:103f78000440bc000281e800a49d2000640379008d
:103f8800611ab80009017800880078000a407800b2
:103f9800060001004f06be004f05be004f04be00dc
:103fa8000080fa00000006000200fa008824ef00f2
:103fb80021cabf000f0032000042eb00e4ff9f005f
:103fc80064a2200014427800f4ff9f00240020001f
:103fd800050020000f81e900a1062000f61907005e
:103fe8001300200012a220001107200021cabf00e0
:103ff800b2ff07006000b8008efe07000080fa00dc
:1040080000000600881f78000244780034c0b3001e
:10401800e1cf40000d003a00e04f54000b003a0099
:1040280085062000850f500003003a00deff0700d8
:104038006a0aa90004003700b5062000850f500061
:1040480002003a006a0aa800084278000440780092
:104058004f04780000000600889fbe008a9fbe00bb
:104068008c9fbe00004578008104780082057800a6
:1040780058518000611eb8000e003700784090004b
:10408800a2c0b3000440bc0064014100a49d20000c
:1040980064037900e00f5300050032000c02be00f3
:1040a8000b017800890078000a40780006000100ba
:1040b80018047800e00f5400f0ff3a004f06be00e5
:1040c8004f05be004f04be0000000600f2874700ff
:1040d800889fbe008a9fbe008c9fbe008e1f7800fe
:1040e800585180002e2aa9002e4aa800c4538000e7
:1040f800b44478000402e800344078008082fb0071
:10410800b44078000183fb004833dd000503430019
:10411800d6b79f000402e800b4427800e5e79f00a4
:104128002442900084ef9f00c4e79f000045eb0005
:104138007e8157000a6978002400200005002000cd
:104148009106200000c0eb009b1907008a4f500021
:1041580003003a0080c2b30022eab7001ac0b300d5
:104168008984fb0009007800780ab4008045eb00d8
:10417800b3003700050078003046780030427800f8
:10418800e94f52000c003a002e2aa800104278008d
:10419800044078001feab70062026200040032009f
:1041a8002e6aab00020032002e4aa9001700370021
:1041b8002e6aa90015003700e44f520013003a0098
:1041c8001047780000027800d4467800d440780080
:1041d800f1e79f0054407800d440780054417800bb
:1041e800e4b79f002ecaab000400320034a22000be
:1041f80014427800a4e79f0009003700fe815700a9
:104208003bfc0700e04f500005003a000c86fb001d
:104218008c84440009007800780ab4008a003700ca
:10422800080278000100370014027800e00f5200fd
:1042380004003200e44290008ecf5200faff3a00a8
:104248000d003700800020008ffa07000002780078
:10425800e00f52000f0032006e429800afe0970066
:10426800714298008002eb00150298002502980020
:10427800080a7800040478006000200084bf9f00ca
:1042880081fa0700000778000fba9700e00f57007f
:104298009a003a006fb297000400e8005f00370008
:1042a8002e0298000c86fb008c844400cc538000be
:1042b800090046008045eb000002eb008802780008
:1042c8000a4478004d0037001045780080067800d1
:1042d80056c0b300dd4f1300040032000a85fb000e
:1042e8008a84440009004600440037002002200068
:1042f80084bf9f00f5b79f0063fa070000037800aa
:10430800dd437800275b98005d407800305b9800bb
:10431800dd4078008183fb0047039800dd4078008a
:104328000180fb004800dd00870340004703980038
:104338009d4390008783fb00270398000fba9700de
:10434800140398001600900000a0a0001003980025
:10435800160090000090a000100398006000b800bc
:10436800000b9800110b9800045b98002fe0970051
:10437800105b9800560890000030b200ffb297001a
:1043880001102000810f500011003a00e08f530007
:1043980002003a001700200027039800a6039000a7
:1043a800f08f530002003600070120002703980011
:1043b800a60390008703e900100020008703dd00b2
:1043c800270398009603900007a0a1001703980000
:1043d800a6039000370398002e009000000b780089
:1043e800260798008b45e8000a85fb008a8444006c
:1043f80009004600e00f530007003200dfb09700c5
:10440800818f5400070031007fe3970086cf550065
:10441800adff390003003700050478001ac0b30067
:10442800020037000845780005047800ffe397008c
:1044380087cf5500020032001ac0b30006003700cb
:10444800e04f550004003a00800278005fb0970002
:10445800808f540047ff3900e00f540016003200e7
:10446800e04f550018003200130037001805780097
:104478000b003700990078001104980003003700fa
:1044880010027800a40498008dfa07002900900013
:10449800e00f5000faff3a000900780088fa070098
:1044a80098049000e08f5400f2ff3a00080078006a
:1044b80083fa07000a047800e00f5400ebff3a0083
:1044c80008407800070037006fe097001eeab70041
:1044d8008fe897000182fb0034518800585188000a
:1044e80010c0b3004f0778004f06be004f05be004e
:1044f8004f04be002f01b100000006009402900096
:10450800050f78002d4798008002eb0025079800da
:104518001e029800e0cf560061ff320061ff3700ad
:104528000200fa00889fbe008a1f7800f8ff270063
:104538001d003700a451800082a32000e20f520022
:1045480004003c000401e8006c11b90085a32000b8
:10455800050141009200780024072000848f500054
:1045680002003200888f500004003a000281e800ff
:10457800a300200021cabf0050fe07006524800068
:104588008c24ef00362aed00a4518000e20f52007f
:1045980003003c000402e800a45188000100370031
:1045a800342aef0065248800b4518000e00f5200df
:1045b800e0ff3a0084508000e10f4200030032001f
:1045c800100af800140af90010aaef0008f02000f9
:1045d800a05080008002640004202000848f5200d4
:1045e8003b01320006003e00e08f52000e00320010
:1045f80004102000848f520011033a00760037001f
:1046080004402000848f5200c30232000410b0001e
:10461800848f5200da02320004302000848f520066
:1046280007033a0059013700a8508000080fb2006c
:10463800f00f54004500320004022000840f54009b
:1046480047003200e00f5400fd023a0056fe070012
:1046580064518000080a78001802980094029000bb
:1046680005a0a00015029800940290000590a000f3
:10467800150298009402900005d0a0001502980039
:104688004501200005129800050420004502980005
:104698006033b800060a9800170a9800285a98004c
:1046a800085a9800d40a90000580a1000590a1003e
:1046b800550a980080c2eb00155a980030c0b30024
:1046c80069eab700084078001eeab7001feab70099
:1046d80020eab7007851880058518800c8508800ef
:1046e80068248800f40f200054248800c0082000a3
:1046f8008224b600d5072000052488008824880075
:104708007424880004a020004822de00c424880005
:1047180084002000a4248800a5002000a524880087
:10472800a4248800040320003424880024002000e6
:104738003425880048258800b8248800aae4a90000
:10474800a404200004258800b8023700a4a620008d
:104758001442780061426200b9023200fa0137005f
:1047680085ff9f0024c3b30094ff9f00240020000e
:1047780005002000688157009106200000c0eb006a
:104788000d180700e04f5000100032001400200000
:10479800442488008ec0a900740680000480a1000b
:1047a8000490a00004a0a000740688009ec0a80081
:1047b80004ff2000a550800005026200700242003c
:1047c800a45088008cc4a8009d0237006a0aa9007a
:1047d8000401200099023700a4508000040fb200a1
:1047e80006022000860f52005700320005003e00e6
:1047f800e00f52000a003200f00f520090023a0017
:104808001200370006032000860f5200870032008e
:1048180005042000850f520089023a00a8003700dd
:10482800a45080006f02620003003200e20f5200c1
:1048380083023a00c4013700140020005424880081
:104848008c04a800b40f200045023700a450800053
:104858006f026200e20f520034003200e40f52008f
:1048680034003200e00f520075023a008051800097
:10487800e00f50000100320091f90700800020008d
:1048880001f9070080518800e00f5000150132003f
:104898001e6aef001f6aef002e2aef0030c0b30037
:1048a80068eab700d400200054258800ac24ef0043
:1048b800ae24ef00b024ef00b224ef00b424ef00e0
:1048c800b624ef00b824ef00ba24ef00bc24ef00b0
:1048d800be24ef00c024ef00c224ef00c424ef0080
:1048e800c624ef00c824ef0094e4ab0006003a00a9
:1048f8002e0aa80000c8b30020eab7000408200068
:10490800b4248800aae4a8009424a8009424a90048
:104918002e8aa9002eaaa9009484a8003403200096
:10492800945088006d0242000f0237009484a90059
:1049380009023700f400200064248800f40f2000e6
:104948008424880039023700a45080006f02620076
:10495800e10f52001300320003003900e20f520049
:1049680037023a001c003700d0538000e00f500097
:104978000200320052f907007a2aef0083518000c2
:1049880004c8b3008449780064c0b3009441980017
:104998000042eb00a441980015c0b300b54198004f
:1049a800b300370066518000160290000420b20060
:1049b8002302320016029000850262008b01320049
:1049c8008451800044429000e94f5200e8013a00c7
:1049d80054c3b300cc0137008851800018427800d6
:1049e8000480fb00a8f80700d0538800e00f5000af
:1049f800bc00320018487800f84290008582fb001d
:104a08006451800045029800080078002cf90700de
:104a180064518000440090009bf807008051880092
:104a2800e00f5000c1003a00ae003700a4508000eb
:104a38006f026200e10f52001900320003003900d2
:104a4800e20f5200fe013a00b8003700188aab00a6
:104a5800fb013a008151800004c8b3008448780003
:104a680064c0b300944098000042eb00a440980052
:104a780015c0b300b5409800c4409800d4409800d1
:104a8800d553800095427800e5409800f44098009e
:104a9800d3538000134078000082fb00c900370020
:104aa80066518000160290000420b200e401320032
:104ab8001602900085026200ad013a004b013700f2
:104ac80061fa0700a0508000000464002c00370041
:104ad800a4508000040fb200d9013a00a65080000b
:104ae8006f036300e10f5300130032000300390025
:104af800e20f5300d2013a001500370010c0b3008e
:104b080021eab700815180008448780055c0b3007d
:104b18009540980015a2200095427800a54098007d
:104b2800b4409800c4409800d4409800e4409800ed
:104b3800f44098002101370064518000140390006c
:104b480085026300be01320014029000250137007f
:104b580074518000610262004722dd0015a2200026
:104b68009542780004c272000440780020eab70039
:104b780030c0b30068eab700a450800004046400a1
:104b88000810b000a8508800ad013700a45080007c
:104b9800040fb20005022000850f520066003200a3
:104ba80005003e00e00f52000d003200f00f5200e9
:104bb800a3013a001c00370005042000850f5200ad
:104bc800d7003200f0824200850f5200e200320026
:104bd80005032000850f520099013a008400370030
:104be800d453800014549000084078006beab70052
:104bf800070037009404900014007800b0f807000c
:104c0800405180000008eb00adf8070049518800ca
:104c180044518000e00f5200f6ff3a00e04f540084
:104c280082013a0037013700a45080006f02620009
:104c3800e10f5200e600320003003900e20f520093
:104c48007f013a00130037008351800004c8b30085
:104c58008449780064c0b300944198006b4aed0021
:104c6800a041980024c0b300b44198000042eb0072
:104c7800c4419800d441980085c0b300e54198002c
:104c8800f441980084002000040178008300780033
:104c98004d00370060002000fbf707000004780093
:104ca800e00f54000f0032008951800063854400f2
:104cb8008984e8001a4278000480fb004800dd007f
:104cc800994278000582fb0004004000eef70700d7
:104cd800000c7800e00f500004003a00080078004b
:104ce80077f8070034c3b300070137001a45780086
:104cf8000a82fb004822dd00994478008982fb0083
:104d080005024200244098004822de003440980002
:104d1800445180001404980048518800c05388000a
:104d2800b5a62000954278004544980030c0b300ed
:104d380068eab7003d013700a45080006f026200a6
:104d4800e10f5200a200320003003900e20f5200c6
:104d58003b013a001f0037008151800004c8b300ae
:104d68008448780064c0b300944098006b4aed0012
:104d7800a040980024c0b300b44098000042eb0063
:104d8800c4409800d4409800445180001402780030
:104d980024429000e44098004451800014027800b6
:104da80034429000f4409800445180009401780007
:104db800a34290008582fb00334290004822dd0028
:104dc80005027200820020006051800033fb07005a
:104dd800e700370030c0b30068eab7006b4aed005f
:104de8006beab7000431200014013a000f013700c4
:104df800a45080006f02620005002000e30f5200fb
:104e0800e08f5a000e013e000460010003003700e5
:104e18002e0037006e0037003a003700c9fa070045
:104e2800e5a1200095427800e0cf520010003a003a
:104e3800280af8006c0af900090037001402780003
:104e4800c4538800a1fc0700e04f500019003a0045
:104e5800bcfa070064538000140290006453880071
:104e680064538000e00f5200f4ff3a00110037004d
:104e780044518000645388000100370014029000f8
:104e8800e00f52000300320044439000854f530066
:104e9800faff3a006453880014027800c45388006b
:104ea8008afc0700e04f500002003a00a5fa07000c
:104eb8006c2aef002e4aab00ad003200645380002c
:104ec800e00f5200aa003a00130037007451800026
:104ed80064026200d5003a002e4aa8008151800081
:104ee8008448780034c0b300944098002e6aab0020
:104ef80001003a0044c0b300a44098000042eb000f
:104f08002800370030c0b30068eab7006453800057
:104f1800e00f5200c5003a0044c3b3007a003700de
:104f280014a22000144278000482fb00050020002f
:104f38000001eb00c107200000c0eb001e160700af
:104f4800e04f5000be003a0004ff2000a05080004f
:104f580000026200b8003700a45080006f026200af
:104f680005002000e30f5200e08f5a00b4003e0015
:104f78000460010003003700150037001d003700ea
:104f88001f003700815180000042eb008448780000
:104f980095c0b30095409800e5a12000954278009f
:104fa800a5409800b4409800c4409800d4409800a8
:104fb800e4409800f44098000002eb008401780077
:104fc8008200200060518000d8fa0700680037008e
:104fd80065518000150290000420b200980032004c
:104fe800150290000410b20061003a00aaf8070008
:104ff8009300370030c0b30068eab7005c003700a0
:1050080004f02000a5508000050262000410b000e2
:10501800a45088002ecaab001300320031a2200031
:105028009140780001407800a2c0b3000440bc0061
:10503800a49d20008202420064027900350190009c
:10504800c501900021cabf0004000100e04f5000d4
:105058001c003a0090c3b30022eab70004502000b5
:10506800a450880017003700585180009ac3b30035
:105078000950200011003700f840900001407800e6
:10508800a2c0b3000440bc00a49d200082024200dc
:105098006402790035019000c501900021cabf0063
:1050a80004000100e04f500003003a000a40780075
:1050b80022eab700a950880018047800e00f5400cd
:1050c800edff3a002eeaab005d00320041a220005d
:1050d8009140780001407800a2c0b3000440bc00b1
:1050e800a49d2000820242006402790035019000ec
:1050f800c501900021cabf0004000100e04f500024
:105108004f003a0094c3b3000440780022eab70085
:105118000450200049003700a4508000040fb2005a
:10512800f00f520046003a00a45080006f0262005f
:10513800e30f520007003200e50f52000e00320064
:10514800e10f52003e003a009444a80054012000a8
:10515800030037009444a9009404a800b400200078
:1051680094508800040420000424880082c4a80005
:10517800142aec0032003700a550880030003700b0
:10518800a4508000040fb2002d003a0085002000d2
:10519800a524880064248800f50f20005524880081
:1051a800c00820008224b600d60720000624880004
:1051b80084248800752488008c04a80024a2200078
:1051c8001442780045c3b300c1c6b300854f5200ee
:1051d8001000320006003e008140e800e74f520010
:1051e8000c00320081c0e8008542e9000600370063
:1051f80051c6b30055c3b300854f520005003200b5
:10520800e9c04000e4c24200854f5200010032006c
:1052180001c7b3008180fb001400200005002000b6
:1052280062a2200021cabf006315070004ff200006
:10523800a55080000502620070024200a450880058
:105248004f0578004f04be000080fa0000000600f9
:10525800e04f500013003a00555180000e0037000f
:10526800150390000900370026029000040037005b
:105278009403900007b0a100170298001402780068
:10528800e00f5200faff3a0016037800e00f5300cf
:10529800f5ff3a0095027800e08f5200f0ff3a00df
:1052a80000000600e3f80700e00f5000030032009a
:1052b8001002900004b0a10014009800000006003d
:1052c8000400fa00889fbe008a9fbe008c1f7800e9
:1052d80001447800824478000305780004067800c9
:1052e80005027800860178008745780065c0b3001c
:1052f80016a2200016437800864f500050003a004e
:1053080007f02000a55080008583630015c0b30016
:1053180006402000868f530049003a0065518000fe
:10532800150390000620b20005c1b3004400320006
:10533800ebcf54001c003a005651800001003700a2
:1053480016037800e00f53003c003200e64290005c
:105358008582fb008c8f5200f9ff3a003e0037002f
:10536800a702900004003700950390000720b200c0
:105378003200320095027800e08f5200faff3a00be
:10538800960290000100370095027800e08f5200e5
:105398002a003200a54390008783fb008a8f5300c0
:1053a800f9ff3a0031003700e1cf54000a003a0013
:1053b800e00f550008003a00e24f540006003e0096
:1053c8000c407800a3bf9f0094bf9f00a0ff070078
:1053d8001fba9700afb997008151800088487800bc
:1053e80099409800aa4098004855de00ba409800b5
:1053f800cc4098004866de00dc409800e440980005
:10540800c822de00f540980060518000afea97009e
:1054180015589800e0cf550004003a00820020009b
:10542800c2f907008b42780005003700820020008f
:105438009af907008042eb000100370035c0b3003d
:10544800054078004f0678004f05be004f04be00a7
:105458000080fa0000000600a603900035c0b300e3
:10546800e08f5300beff3a00f5ff37002503980090
:10547800d9ff370075518000e1826200d4cdb300b6
:1054880001003a00d4c5b300b6508000d60a900097
:105498000530b20001003a000444a100d60a900089
:1054a8000530b20006102000868f520001003a0035
:1054b8000404a1000482fb005425880004a22000f3
:1054c800144278000482fb00b42488008180fb0029
:1054d800c408dd00f007b20000807000f0248800e6
:1054e800188aa80000000600e94f50000f003a0093
:1054f800745180007002620045a0200001003a004b
:1055080005a02000765180004433de000683ea00bf
:10551800610363004433dd00745180000440a1003e
:10552800060272007451880023003700745180000d
:105538000402b200c5a0200001003a00e482520033
:10554800765180004533de000683ea00610363007c
:105558004533dd00745180000450a100060272003a
:1055680074518800ed4f500013003a00b450800089
:10557800740090000409900094099000440390007e
:10558800010020000200500083805800070020001e
:10559800860f5000878f58000200360044039000a1
:1055a8002300370074009000040b9000940b9000c7
:1055b800060350001e003700b4508000540b9000c2
:1055c8000630b20007102000870f530005003a008c
:1055d800e94f50000e003200040b9000940b90002d
:1055e8003b00370054019000e4019000040890004b
:1055f80094089000440390000000510081805900f5
:1056080007002000860f5000878f580002003600e0
:10561800440390002e00370054009000e4009000ee
:10562800040b9000940b90000603500028003700ec
:10563800240a90000d003700b40b9000340a900043
:10564800144090000080fb000000e8006600b900ec
:10565800e70378009702980005003700b40b900024
:105668000408900094089000008243009402980077
:105678000042eb0094429800f63fb20004c02f00ad
:105688001502620006027200840a7800b750800092
:10569800170090004b00de00610060004e00dd0046
:1056a80004e0a10000027200840a780097039000c9
:1056b800ca3bde00e1836300cb3bdd0004b0a10000
:1056c8000702720004f0a000840a780000000600b7
:1056d800d40b90000730b20000102000808f5300d8
:1056e800deff3a00d4ff3700889fbe008a9fbe00c5
:1056f8008c9fbe008e1f7800a4508000c950800087
:10570800f08464006a013a00ca50800061056500af
:10571800c5003a000a4078004ef80700e04f5000f4
:10572800c0003200b8508000085a9000040fb20040
:1057380005022000850f520022003200f08242004c
:10574800850f52003b003200f00f520051013a0021
:10575800085a90006f026200e10f520009003200ff
:1057680003003c00e00f52004600320049013700b8
:10577800e20f520011003200ef0f520045013a00cb
:1057880078003700080890009808900050049800a6
:10579800610498001802900004b0a0001404980056
:1057a80090c0b30050ff07002858900091c0b30084
:1057b80030ff0700180aa8003d0137000a5c98006e
:1057c80044003700085a90006f026200cfa2de0042
:1057d800046001002b003700f1ff37000d0037008f
:1057e8003a0037002b0137002a013700290137001a
:1057f8002801370027013700260137002501370027
:105808002401370023013700220137002101370026
:1058180054003700080a9000980a90005404980031
:10582800650498001802900004b0a00014049800c1
:105838001c003700085a90006f026200cfa2de00f9
:10584800046001000f003700160037001a00370007
:105858001e0037000f0137000e0137000d01370019
:105868000c0137000b0137000a0137000901370026
:105878000801370007013700060137000501370026
:10588800380037001802900004b0a10014049800f2
:10589800d0c0b30014ff070028589000d1c0b3004f
:1058a800c3ff370010c0b3000fff0700285890004f
:1058b80011c0b300beff3700080a9000980a900094
:1058c8005404980065049800b2ff37000042eb00ca
:1058d800045c9800180290000490a000140498003a
:1058e800b4518000e30f52004b003c000402e80072
:1058f800b451880094518000e20f520003003c002c
:105908000402e8009451880001003700322aef00b1
:10591800955180006c2bb9000602780027072000fb
:1059280086a3200007337a000683e80004034300b7
:105938000808900098089000008bbe008502e800d7
:105948006c2bb90025a32000b808900081327b0099
:10595800ee824200848242000043eb0096429800a7
:10596800240037000042eb00045c98001802900005
:105978000490a00014049800b4518000e30f520072
:1059880025003c000402e800b451880094518000ce
:10599800e20f520003003c000402e8009451880022
:1059a80001003700322aef00955180006c2bb900b6
:1059b80006027800f7ff270086a3200007337a0045
:1059c8000683e80004034300000beb00361378005d
:1059d8008502e8006c2bb90025a3200086824200ce
:1059e800800aeb0005a4200084824200c858900079
:1059f80091429800285b9000864a780025a42000f0
:105a08000482420038589000004a7800185c9000e0
:105a1800184298000200370084c0b300345c980034
:105a28008044eb00180aa800182aab008e00320048
:105a38009f003700b8508000085a9000040fb20049
:105a480005042000850f520004003200f082420055
:105a5800850f52007a003a0012003700085a900069
:105a68006f026200e10f520009003200ef0f52008e
:105a780046003200e00f520071003a0090c0b300b7
:105a880099fe07002858900091c0b3001100370014
:105a98000042eb00045c9800a800900031049800d4
:105aa80012003700085a90006f026200e10f52009e
:105ab8000a003200ef0f520034003200e00f5200ab
:105ac8005f003a0010c0b30087fe07002858900016
:105ad80011c0b30067fe0700750037000042eb00f5
:105ae800045c980028029000340498001802900082
:105af8000490a00014049800b4518000e30f5200f1
:105b08004a003c000402e800b45188009451800027
:105b1800e20f520003003c000402e80094518800a0
:105b280001003700322aef00955180006c2bb90034
:105b3800060278002607200086367a00040346000d
:105b48000808900098089000008bbe008502e800c5
:105b58006c2bb90025a32000b808900081327b0087
:105b6800848245000043eb0096429800285b900031
:105b7800864a78000402450038589000004a7800a8
:105b8800185c9000184298002a0037000042eb0089
:105b9800045c9800a8009000310498001802900056
:105ba8000490a00014049800b4518000e30f520040
:105bb8001e003c000402e800b451880094518000a3
:105bc800e20f520003003c000402e80094518800f0
:105bd80001003700322aef00955180006c2bb90084
:105be800060278008e367a0004034600000beb00ac
:105bf800361378008502e8006c2bb90025a3200035
:105c080086824200800aeb0084824500485b90004f
:105c18009642980028589000804a7800040245006f
:105c2800b8589000014a7800d5ff370084c0b30007
:105c3800345c9800e0cf54001000320001003700b7
:105c480019c0b300b45080008042eb00055a980098
:105c5800a402900035029800940290000590a000dc
:105c680015029800050037008da320000d86e80076
:105c7800e60546000b85e800feff270030c0b300ac
:105c8800f4f60700e04f50006aff3a00182aa8000f
:105c9800070037000042eb00045c980018029000ef
:105ca8000490a0001404980019c0b3005dff3700e9
:105cb8004f0778004f06be004f05be004f04be00d8
:105cc8000000060064518000140290000420b20015
:105cd80010c0b30014003200505180000e0037008d
:105ce8001002900009003700a40290000400370059
:105cf800150390000620b2000a00320095027800d1
:105d0800e08f5200faff3a0014027800e00f5200c8
:105d1800f5ff3a0010007800e00f5000f0ff3a005d
:105d28000000060010c0b30000000600881f7800bd
:105d38000144780064c0b30015a2200095427800a1
:105d4800854f500014003a0006f02000a050800053
:105d58000003630014c0b30005402000850f530002
:105d68000d003a00d7ff07000043780024c0b300b5
:105d7800e04f530008003a00084078001eeab700d8
:105d880080c2eb0064518000155a9800043320004b
:105d9800a450880006427800044078004f04780038
:105da800000006008ec0a90082c4ab0012003200b9
:105db80080c4ab00100032000404200004248800d2
:105dc80094508000e00f52000b003200122aed00c0
:105dd80094508000e00f520007003a0082c4a900e6
:105de80004f02000a050800000026200e00f520082
:105df80001003200142aec008cc4ab000b00320006
:105e08008ac4ab00090032008cc4a9000404200035
:105e180054248800a550800070025200848f5200dc
:105e280002003a0004102000845088008c04ab0063
:105e3800060032008a04ab0004003200140020007f
:105e4800542488008c04a900102aef008c64ab004d
:105e5800c50032008a64ab00c30032008c24ab005a
:105e6800080032008a24ab0006003200b4508000db
:105e7800540a90000430b20005102000850f52002b
:105e8800b9003a00188aa9009624800084002000ee
:105e980054248800b4508000a45a9000f72480004d
:105ea80085826b00ef826200ae003a00e802630070
:105eb80064036300e08f52000200320085a02000d6
:105ec8000100370005a02000e00f53000100320058
:105ed800e482420006c02300150363000780200007
:105ee800870f530029003a00f63f2000150363008e
:105ef800040890009408900006004000e0804800e4
:105f0800000a9800110a98008002eb00750a9800b0
:105f180094039000cb3bde008783ea00e1836300b3
:105f2800cb3bdd009402900005b0a100878272008f
:105f380015029800845a9000f0cf520008003200f1
:105f4800845b900005c2b30085cf53000400320083
:105f5800845b9000f0c2420085cf530024003a00d1
:105f68000408900094089000740390000700200033
:105f7800860f5000878f58007a0039006033b800c8
:105f8800060a9800170a98005300370007c0200037
:105f9800870f53000300320007c02200870f530009
:105fa80023003a00f63f2000150363000408900020
:105fb8009408900006004000e0804800000a98001d
:105fc800110a98008002eb00750a9800940390006b
:105fd800cb3bde008783ea00e1836300cb3bdd0037
:105fe8009402900005b0a100878272001502980003
:105ff800d40a90000530b20007102000878f5200a5
:1060080032003200c4029000850f53002f0039007f
:10601800040890009408900054039000e403900052
:10602800860f5000878f58004e0039002700370030
:1060380005802200850f53002a003a009402900040
:1060480005c0a00015029800f40a90008502e80037
:10605800750a9800d40a9000c82ade00e38262001c
:10606800e28f520008003200e38f52000300320032
:10607800e18f520004003a0014003700a45a90003f
:10608800e0cf5200110035001403900005002200f3
:106098008502630033003200740b90008412900074
:1060a800850f53002f003600940290000560a00071
:1060b8001502980075c1b300455a9800845a90009b
:1060c800f540b300055a9800260037009402900066
:1060d8000580a00015029800845a90008542e800c7
:1060e800f8ff370005802300850f530005003a00ac
:1060f800940290000550a0001502980015c1b30045
:10610800edff3700140390000643e8007f036300a7
:106118009403900005fe2f0085826300868272003a
:106128001502980094029000ff826200f38f5200db
:106138000c003400940290000560a000150298003d
:1061480035c1b300455a9800845a9000f540b30011
:10615800055a9800f40f20007424880024002000b9
:106168005424880060fd07008c44ab0029003200ed
:106178008a44ab00270032004400200054248800e1
:10618800555180000030200007102000180037000b
:1061980025029000e00f5200140032002402900003
:1061a80010003700540b90000630b200800f5300e7
:1061b80002003200870f530006003a0034039000b3
:1061c800e00f530003003200340390000603e90097
:1061d800360298001403900006c0a1001602980029
:1061e80014027800e00f5200eeff3a0095027800a2
:1061f800e08f5200e6ff3a00180aa900182aa90001
:10620800184aa900186aa900054078001aeab700d8
:1062180035fd07008c24ab003b0032008a24ab001c
:1062280039003200188aa900b4508000d40a9000be
:106238000530b20006102000868f52002e00320072
:10624800140390000643e8007f0363009403900062
:1062580005fe2f0085826300868272001502980071
:1062680094029000ff826200f38f520022003400f3
:106278008ee4ab000200320005c2b300455a980014
:106288008ea4ab000200320015c2b300455a980034
:106298008e84ab000200320025c2b300455a980034
:1062a8008e64ab000200320035c2b300455a980034
:1062b8008e44ab000200320045c2b300455a980034
:1062c8008e24ab000200320055c2b300455a980034
:1062d8008e04ab000200320065c2b300455a980034
:1062e800940290000560a00015029800845a90005e
:1062f800f540b300055a9800f40f20007424880074
:1063080024002000542488000000060094408000e7
:10631800e20f520002003a00340020009440880046
:1063280000000600a44f8000b54f8000864d210074
:10633800860f5200e08f5a0045003a00c44f800093
:10634800d54f800077d02c00870f5200e08f5a007d
:106358003f003a00f49f200014427800e04f5200ba
:1063680019003a00b4408000660242009442780066
:1063780061c36200610363004833dd0005408000ab
:106388000580a100068372000640880094437800c7
:106398008782fb00c82add000520b2000690a10014
:1063a8008502730005408800144278000482fb00cf
:1063b8004422de00610262004a22dd0005a0a1003d
:1063c800848272000540880045418000e08f5200b9
:1063d8000300320064418000e00f520002003a00de
:1063e8000088a800010037000088a900f40f2000e9
:1063f800848f52000300320065418000848f520070
:1064080002003a0000a8a8000100370000a8a9006f
:1064180055418000e08f5200030032007441800033
:10642800e00f520002003a0000c8a800010037003f
:1064380000c8a900f40f2000848f52007c003200ad
:1064480075418000848f52007b003a007800370045
:1064580005408000e80f500035003c00564580009c
:10646800610363004833dd000580a1008682720065
:1064780064458000610262004922dd000590a100a8
:106488000482720075458000e1826200ca2add003c
:1064980004a0a10005027200044088000168a90058
:1064a8000188a90001a8a900b44580006102620022
:1064b8004522dd00154080000550a10004827200cd
:1064c800c5458000e1826200c62add000460a100a3
:1064d800050272001440880044418000e00f520019
:1064e80002003a000088a800060037000088a900ca
:1064f800f50f2000850f520002003a0000a8a800fe
:106508000100370000a8a90054418000e00f5200a4
:1065180002003a0000c8a8004700370000c8a900d8
:10652800f50f2000850f520041003200420037006d
:1065380026468000610363004833dd000580a10022
:106548008682720034468000610262004922dd00c2
:106558000590a1000482720015468000e182620065
:10656800ca2add0004a0a1000502720004408800c8
:106578000168a9000188a90001a8a9005445800064
:10658800610262004522dd00154080000550a1002f
:106598000482720085458000e1826200c62add001f
:1065a8000460a10005027200144088004441800084
:1065b800e00f520003003200c5458000e18f520011
:1065c80002003a000088a800010037000088a900ee
:1065d800f50f2000850f520003003200a44580000b
:1065e800e10f520002003a0000a8a800010037009d
:1065f80000a8a90054418000e00f520003003200b7
:1066080095458000e18f520002003a0000c8a800ba
:106618000100370000c8a900f50f2000850f5200bf
:1066280003003200b4458000e10f520002003a0036
:1066380000e8a8000000060000e8a9000000060025
:10664800a44f8000b54f8000864d2100860f520070
:10665800e08f5a004a003a00c44f8000d54f8000ae
:1066680077d02c00870f5200e08f5a009f003a0025
:10667800f49f200014427800e04f520030003a00a6
:10668800b4408000660242009442780061c3620010
:10669800610363004833dd00054080000580a100e8
:1066a8000683720006408800944378008782fb00c6
:1066b800c82add000520b2000690a10085027300fb
:1066c80005408800944378000783fb004333de00cd
:1066d800610363004b33dd0005b0a10086827200c0
:1066e80005408800944378000783fb004433de00ac
:1066f800610363004a33dd0005a0a10086827200b1
:1067080005408800944378000783fb004633de0089
:10671800610363004c33dd0005c0a100868272006e
:1067280005408800144278000482fb004722de00fe
:106738004d22dd0005d0a10084827200054088004a
:10674800b640800067034300964278000582fb004c
:106758004322dd000402b200154080000550a1006c
:106768008482720015408800164378000682fb0078
:106778004322dd000404b2000560a10037003700a1
:10678800f6e82000860f5200e08f5a0057003a00c2
:10679800c44f8000d54f8000e30f5200e08f5a00ad
:1067a80052003a00f49f200014427800e04f520053
:1067b80020003a0074458000610262004822dd0032
:1067c800054080000580a100048272008745800092
:1067d800e1836300c93bdd000490a10087037200d8
:1067e80066458000610363004a33dd0007a0a1000d
:1067f8000683730055458000e1826200cb2add00e4
:1068080006b0a10085027300944580006102620011
:106818004c22dd0005c0a10004827200a54580005d
:10682800e1826200cd2add0004d0a10005027200d9
:1068380004408800d4458000610262004522dd00e2
:10684800154080000550a10004827200e5458000d3
:10685800e1826200c62add000460a1000502720020
:106868001440880045418000e08f52000300320048
:1068780064418000e00f520002003a000088a8003e
:10688800010037000088a900f40f2000848f52000f
:106898000300320065418000848f520002003a00f4
:1068a80000a8a8000100370000a8a90055418000f1
:1068b800e08f52000300320074418000e00f520064
:1068c80002003a0000c8a8000100370000c8a9006b
:1068d800f40f2000848f52009b0032007541800025
:1068e800848f52009a003a0097003700f49f2000e6
:1068f80014427800e80f500044003c00e04f52007a
:1069080020003a0064458000610262004822dd00f0
:10691800054080000580a100048272005745800070
:10692800e1836300c93bdd000490a1008703720086
:1069380076458000610363004a33dd0007a0a100ab
:106948000683730085458000e1826200cb2add0062
:1069580006b0a100850273009445800061026200c0
:106968004c22dd0005c0a10004827200a54580000c
:10697800e1826200cd2add0004d0a1000502720088
:1069880004408800b4458000610262004522dd00b1
:10699800154080000550a10004827200c5458000a2
:1069a800e1826200c62add000460a10005027200cf
:1069b8001440880044418000e00f520002003a0071
:1069c8000088a800060037000088a900f50f2000fd
:1069d800850f520002003a0000a8a8000100370005
:1069e80000a8a90054418000e00f520002003a00bc
:1069f80000c8a8005600370000c8a900f50f2000fd
:106a0800850f52005000320051003700e04f52000d
:106a180020003a0034468000610262004822dd000e
:106a2800054080000580a10004827200274680008e
:106a3800e1836300c93bdd000490a1008703720075
:106a480016468000610363004a33dd0007a0a100f9
:106a58000683730045468000e1826200cb2add0090
:106a680006b0a10085027300f4458000610262004f
:106a78004c22dd0005c0a10004827200054680009a
:106a8800e1826200cd2add0004d0a1000502720077
:106a98000440880054458000610262004522dd0000
:106aa800154080000550a1000482720085458000d1
:106ab800e1826200c62add000460a10005027200be
:106ac8001440880044418000e00f52000300320067
:106ad800c5458000e18f520002003a000088a800f6
:106ae800010037000088a900f50f2000850f52002b
:106af80003003200a4458000e10f520002003a0072
:106b080000a8a8000100370000a8a900544180008f
:106b1800e00f52000300320095458000e18f5200db
:106b280002003a0000c8a8000100370000c8a90008
:106b3800f50f2000850f520003003200b445800095
:106b4800e10f520002003a0000e8a8000000060029
:106b580000e8a90000000600889fbe00c49f20002e
:106b6800144278008442e900e1cf52000400360064
:106b7800e44f520002003200e54f520014003a0080
:106b8800e38120006a814100c1408000b04080005c
:106b980006070700c38320006a814100c1408000c6
:106ba800b040800001070700e38620006a814100a9
:106bb800c1408000b0408000fc060700038a200026
:106bc8006a814100c1408000b0408000f70607009c
:106bd800fc49ed00e14f5000ac003e00e49f20006e
:106be80014427800e04f520049003a00aac8bf009a
:106bf80061406000e1036000c83bdd0004408000a4
:106c08000480a10087037200664580006103630069
:106c18004933dd000790a1000683730075458000a5
:106c2800e1826200ca2add0006a0a1008502730085
:106c380084458000610262004b22dd0005b0a1009e
:106c48000482720095458000e1826200cc2add0052
:106c580004c0a1000502720004408800c222ab00f3
:106c68000a0032000410b20008003200844b800091
:106c7800954b8000e40f5200e08f5a002400360044
:106c880061025200e0825a000b003700c222ab00ba
:106c9800160032000128ab0014003200844b80003b
:106ca800954b8000f40f5200e08f5a0018003e0008
:106cb80061024200e0824a00844b8800954b8800bc
:106cc800840078008002200079110700200020004d
:106cd800a511070000e0230091042000ad11070072
:106ce800200020009c110700090037009d0d0700b7
:106cf800004080004900de0061406000a00d0700f0
:106d0800004080004a00de0061406000a90d0700d5
:106d1800464180005640880050418000604088000d
:106d28003482200014427800ef4f520026003e00c3
:106d38000482fb008403e90087b2de00e18262007e
:106d48000f003200840278001200200003002000a7
:106d58000204be00850078008100e90003003300ca
:106d68000804440089844c00fbff370008037300c3
:106d78008502e800ef8f5200f5ff34005640880086
:106d88008783de00e18363000f00320065408000e6
:106d980016002000070020000600be00040178004d
:106da8000201e90003003300000040008180480030
:106db800fbff3700808272000402e800ef0f5200e8
:106dc800f5ff340065408800824b800061408000f8
:106dd80050408000060e0700344280004541800084
:106de800850f520007003a00554180004642800056
:106df800850f530003003a004a08f8000408f90018
:106e080001003700244088001484200014427800d0
:106e1800ef4f520014003e00254080000482fb0022
:106e28000403e90006abde00610363000e003200d4
:106e380016002000070020000600be0004017800ac
:106e48000201e9000300330000004000818048008f
:106e5800fbff3700808272000402e800ef0f520047
:106e6800f5ff34002540880024408000e00f5200e0
:106e780002003400140020002440880024408000d0
:106e8800e00f520001003d0004a8ef00c49f20005d
:106e98001442780064425200e14f52005e003e0006
:106ea800244b8000354b8000e00f5200e08f5a00e1
:106eb80003003a00004580001afd0700050037006e
:106ec800e10f5200e08f5a0002003a0000458000ae
:106ed800dbfd0700c222ab002f003200264b8000ea
:106ee800374b800061024300e0824b00244b88004e
:106ef800354b8800e10f5200e08f5a00020036003f
:106f08006429ef006629ef00200020001611070011
:106f180000002500310c20001e1107000004eb00c2
:106f28000b003700200020000b11070000402d0047
:106f38000103200017110700200020000a11070094
:106f480000402d0001032000121107000804e8008a
:106f5800244b8000354b80006140b900610342003a
:106f6800e0834a00860f5000878f5800edff3900f4
:106f780084007800a0002000cd1007000000250044
:106f8800310c20000311070020002000f210070038
:106f980002a8a90002c8a900f49f200014427800a2
:106fa800e04f52000c003a00004080004800de002c
:106fb80061406000eb0c0700004080004900de00e3
:106fc80061406000ee0c0700004080004a00de00cf
:106fd80061406000f70c0700004080004500de00bb
:106fe80061406000150d0700004080004400de008d
:106ff800614060000a0d0700004080004700de0085
:10700800614060001b0d0700004080004600de0064
:1070180061406000100d07004f04be00000006002c
:107028000002eb00944088000440780014e8b700a0
:10703800b44088001ce8b700000006000200fa000f
:107048001cc8bf0003003a00de0307001ce8b700b5
:107058000c003700b103070024c5b300844f50006b
:1070680008003a001228ef001c68ef001468ef00cf
:10707800b0408000e00f50000200320090ef07009f
:107088001628ef009440800005002000e40f52000d
:10709800e08f5a004f003e000460010004003700f2
:1070a800080037002700370029003700350037006f
:1070b80020002000ac100700fc69ef00140020003d
:1070c8003f0037001cc8bf0042003200930307008e
:1070d800c4c5b300844f50003e003a000000eb00e6
:1070e800801007002400200094408800a20020009f
:1070f80003002000a0182300560f0700d453800077
:10710800844a90008582fb00144b90004833dd00d0
:107118000503730007002000a64f8800b74f8800ba
:10712800a44a90008582fb00344a90004822dd0082
:107138000502720005002000c44f8800d54f880062
:1071480024003700200020008310070021003700aa
:10715800b4408000e38120009341780062822000df
:107168001241780001822000914078001cc8bf00bd
:10717800aa03070044002000e04f5000100032002e
:10718800140037000f01e9008f80e9001cc8bf0018
:10719800dc030700e04f50000e0032006ffa970042
:1071a800e04f520005003a00fffa97008582fb0085
:1071b800f4408000848f5200030032002400200035
:1071c8009440880003003700240020009440880081
:1071d80061fe07000080fa0000000600e68747000d
:1071e800889fbe008a9fbe008c9fbe008e1f7800bd
:1071f80049812000994478000040eb0080cf54007a
:1072080057013a002449800064409000a2c0b300ae
:107218000440bc00020078003009b40040409000ef
:10722800fce9b700fcc8bf00e0ef9f000945780003
:10723800094778008945780009467800894678002a
:10724800200137000d83fb00e402200004b3b900dd
:10725800060078002a09b40000047800c49f2000c2
:10726800144278000443e900e14f530069003e00ee
:1072780018027800e00f520011013a00281390001c
:10728800b8139000e60f5300e08f5b005a003a00f5
:1072980018039000e10f530009013a00e04f56002f
:1072a8002d003a00e0cf55002b003a000868900006
:1072b800986b900086498000050320001103200088
:1072c8000e003700a2c0b3000440bc000201430016
:1072d80022019000850f510003003200810f5100f8
:1072e80004003a00020037001cc0b3000100370058
:1072f8001bc0b3000442e8000040e800874f52007a
:10730800f0ff3900c85a90000580fb004300dd00fb
:107318002c09b40010029000670242004322de00ec
:10732800f4408800685a90000482fb0004418800f9
:107338002860900022e8b7007858900023e8b7004a
:107348000860900024e8b70085bf9f007605070015
:1073580026e8b7008fba9700e04f5500d8003a00ea
:1073680008689000986b9000864980000a4278006f
:107378008503200009003700a2c0b3000440bc0008
:1073880002014300a2009000858f500001003a00de
:107398001ac0b3000442e8000040e800874f5200da
:1073a800f5ff3900c85a90000580fb004300dd0056
:1073b8002c09b40010029000670242004322de004c
:1073c800e4418800685a90000482fb00f441880078
:1073d8002860900040e8b7007858900041e8b7006e
:1073e8000860900042e8b70085bf9f004e0507007f
:1073f80044e8b700b1003700e20f5300e08f5b00ac
:10740800af003a0018029000e90f5200ac003a00b1
:107418009600370064425200e14f5200a8003e0037
:1074280018027800e00f5200a5003a0028139000d7
:10743800b8139000e20f5300e08f5b00a0003a0001
:1074480018039000e10f530086003a00e04f560001
:1074580034003a00e0cf550032003a00e04f5700c0
:1074680030003a0008689000986b900086498000c8
:107478000503200011032000230320001200370019
:10748800a2c0b3000440bc000201430022019000e6
:10749800850f510005003200810f510005003200b0
:1074a800830f510005003200050037001cc0b300ef
:1074b800030037001bc0b300010037001ec0b30033
:1074c8000442e8000040e800874f5200ecff390012
:1074d800c85a90000580fb004300dd002c09b40069
:1074e80010029000670242004322de00f440880048
:1074f800685a90000482fb000441880028609000cc
:1075080022e8b7007858900023e8b7000860900098
:1075180024e8b70085bf9f000305070026e8b700e9
:107528008fba9700e04f550026003a00086890008f
:10753800986b9000864980000a42780085032000f5
:1075480009003700a2c0b3000440bc000201430098
:10755800a2009000858f500001003a001ac0b300c5
:107568000442e8000040e800874f5200f5ff390068
:10757800c85a90000580fb004300dd002c09b400c8
:1075880010029000670242004322de00e4418800b6
:10759800685a90000482fb00f4418800286090003b
:1075a80040e8b7007858900041e8b70008609000bc
:1075b80042e8b70085bf9f00db04070044e8b70036
:1075c8008fba9700e0cf54003d003a000868900059
:1075d800986b900086498000094278009503200046
:1075e80009003700a2c0b3000440bc0002014300f8
:1075f800a2009000858f500001003a0019c0b30026
:107608000442e8000040e800874f5200f5ff3900c7
:10761800c85a90000580fb004300dd002c09b40027
:1076280010029000670242004322de007443880083
:10763800685a90000482fb00844388002860900008
:1076480072e8b7007858900073e8b70008609000b7
:1076580074e8b70085bf9f00b304070076e8b70059
:1076680016003700e90f530015003a00c85a900079
:107678000580fb004300dd002c09b40010029000d7
:10768800670242004322de0004458800685a9000e1
:107698000482fb001445880028609000a4e8b70025
:1076a80078589000a5e8b70008609000a6e8b700f1
:1076b80085bf9f009c040700a8e8b7008fba970011
:1076c8008d46e8006fe9970082cf5600ddfe39004d
:1076d800d48f200014427800e04f52001f0032007f
:1076e8000580fb004300dd002c09b4001000900069
:1076f800670040004300de00c040880062ed0700dc
:10770800b0408800d208f8001a08f900e04f560087
:107718000200320010c0b30014e8b700e0cf5500f3
:107728000200320010c0b30014e8b700e04f570061
:107738000200320010c0b30014e8b700e04f550053
:107748000200320010c0b30014e8b700e0cf5400c4
:107758000200320010c0b30014e8b70014c8bf001c
:107768004f0778004f06be004f05be004f04be000d
:107778006f00b1000000060000a0fe003600f8000f
:10778800849fbe00869fbe00889fbe00692480003b
:107798008c24ef001816800062046400b8003a00d8
:1077a800244b8000354b8000e10f5200e08f5a00d7
:1077b800b3003a00c49f200014427800644252008b
:1077c800e14f5200ae003e0010c0b300ffe9b70021
:1077d800c902a800c8e2a900c9c2a900c9e2a90053
:1077e800c8a2a800044080004922de000482ea0002
:1077f80061026200e1026200c72bdd0066168000ac
:107808000670a10007037300661688004e2bdd0082
:107818006516800005e0a100868272006516880062
:10782800cf22dd006416800004f0a100050272007a
:1078380064168800de0b0700044080004822de0042
:107848000482ea0061026200e1026200c72bdd00e7
:10785800661680000670a10007037300661688008c
:107868004e2bdd006516800005e0a10086827200bf
:1078780065168800cf22dd006416800004f0a100a0
:107888000502720064168800c90b070004408000d6
:107898004a22de000482ea0061026200e10262001c
:1078a800c72bdd00661680000670a1000703730071
:1078b800661688004e2bdd006516800005e0a100e5
:1078c8008682720065168800cf22dd00641680006b
:1078d80004f0a1000502720064168800b40b0700ca
:1078e800044080004b22de000482ea00610262004c
:1078f800e1026200c72bdd00661680000670a10059
:1079080007037300661688004e2bdd00651680009d
:1079180005e0a1008682720065168800cf22dd008e
:107928006416800004f0a100050272006416880045
:107938009f0b0700044080004d22de000482ea000d
:1079480061026200e1026200c72bdd00661680005a
:107958000670a10007037300661688004e2bdd0031
:107968006516800005e0a100868272006516880011
:10797800cf22dd006416800004f0a1000502720029
:10798800641688008a0b0700044080004c22de0041
:107998000482ea0061026200e1026200c72bdd0096
:1079a800661680000670a10007037300661688003b
:1079b8004e2bdd006516800005e0a100868272006e
:1079c80065168800cf22dd006416800004f0a1004f
:1079d8000502720064168800750b070014408000c9
:1079e8004622de000482ea0061026200e1026200cf
:1079f800c72bdd00661680000670a1000703730020
:107a0800661688004e2bdd006516800005e0a10093
:107a18008682720065168800cf22dd006416800019
:107a280004f0a1000502720064168800600b0700cc
:107a3800cce2a800cdc2a800cde2a8005c0b0700ec
:107a4800cce2a900cdc2a900cde2a900580b0700dd
:107a5800cce2a800cdc2a800cde2a800540b0700d4
:107a6800c902a800c8e2a800c9c2a800c9e2a800c3
:107a7800c8a2a80008407800ffe9b700bb0037009b
:107a88001816800062046400b8003a00fc49ed0052
:107a9800e14f5000b5003e0010c0b300fee9b7004a
:107aa800c902a800c8e2a900c9c2a900c9e2a90080
:107ab800c8a2a800044080004922de000482ea002f
:107ac80061026200e1026200c72bdd0066168000d9
:107ad8000670a10007037300661688004e2bdd00b0
:107ae8006516800005e0a100868272006516880090
:107af800cf22dd006416800004f0a10005027200a8
:107b0800641688002a0b0700044080004822de0023
:107b18000482ea0061026200e1026200c72bdd0014
:107b2800661680000670a1000703730066168800b9
:107b38004e2bdd006516800005e0a10086827200ec
:107b480065168800cf22dd006416800004f0a100cd
:107b58000502720064168800150b070004408000b7
:107b68004a22de000482ea0061026200e102620049
:107b7800c72bdd00661680000670a100070373009e
:107b8800661688004e2bdd006516800005e0a10012
:107b98008682720065168800cf22dd006416800098
:107ba80004f0a1000502720064168800000b0700ab
:107bb800044080004b22de000482ea006102620079
:107bc800e1026200c72bdd00661680000670a10086
:107bd80007037300661688004e2bdd0065168000cb
:107be80005e0a1008682720065168800cf22dd00bc
:107bf8006416800004f0a100050272006416880073
:107c0800eb0a0700044080004c22de000482ea00f0
:107c180061026200e1026200c72bdd006616800087
:107c28000670a10007037300661688004e2bdd005e
:107c38006516800005e0a10086827200651688003e
:107c4800cf22dd006416800004f0a1000502720056
:107c580064168800d60a07000488d5000082ea0066
:107c680061026200e1026200c72bdd006616800037
:107c78000670a10007037300661688004e2bdd000e
:107c88006516800005e0a1008682720065168800ee
:107c9800cf22dd006416800004f0a1000502720006
:107ca80064168800c20a0700244080000482ea00a3
:107cb80061026200e1026200c72bdd0066168000e7
:107cc8000670a10007037300661688004e2bdd00be
:107cd8006516800005e0a10086827200651688009e
:107ce800cf22dd006416800004f0a10005027200b6
:107cf80064168800ae0a0700cce2a800cdc2a8002e
:107d0800cde2a800aa0a0700cce2a900cdc2a900ca
:107d1800cde2a900a60a0700cce2a800cdc2a800bf
:107d2800cde2a800a20a0700c902a800c8e2a8007c
:107d3800c9c2a800c9e2a800c8a2a80028408800b3
:107d480008407800fee9b700fde9b7000040800070
:107d58004800de00614060008209070000408000a2
:107d68004900de0061406000850907006924880039
:107d78008660a9004f04be004f03be004f02be003c
:107d88003600f9000080fe0000400600881f7800d9
:107d9800a493200014427800804f52000f003a004c
:107da8000a00370046ec07004029ef0003003700bf
:107db8001004780042ec0700e8538800e053800084
:107dc800e00f5000faff3a0004003700004a800034
:107dd800e00f5000f3ff3a00f8ff37004f04780037
:107de80000000600889fbe008a9fbe000085fb0039
:107df800c802200008d4b9006e024400699320002c
:107e080069027a000402d100614262002a0032004d
:107e18007482440008024200004aeb000402200079
:107e28000902420008024200004aeb00a4022000b6
:107e38000802420069427a00640544008a824400cc
:107e480095429000851f78008043eb000003eb000b
:107e5800860278000482fb008601780000c1eb00ee
:107e680011c2b30069407d0015f507008f87e9004e
:107e780070824400e04f50000b00320008044200ba
:107e880074c5b300044c780044c0b300144498008f
:107e98006022b8000001eb002126200069407d0027
:107ea800450a07001a0037000804420074c0b300ee
:107eb80014449800160037007002440069427a00a2
:107ec80064044400e04f520004003a006022b80005
:107ed8000001eb00e1252000030037006022b80014
:107ee8000001eb002126200069407c00320a0700cf
:107ef800c402200004d5b900649420000a0242009c
:107f08007205450065932000e5427d001542980002
:107f18004f05be004f04be000000060080427800f6
:107f2800a49320001442780020c5b300854f520066
:107f38001d003a001d003700749420001442780098
:107f48000482fb000500200061025200e0825a0012
:107f5800e80f5200e08f5a0010003e000460010054
:107f6800080037000d003700060037000d00370005
:107f78000a003700090037000600370005003700ff
:107f880002003700a0c5b30000000600d0c5b3004a
:107f980000000600e0c5b3000000060090c5b3006d
:107fa80000000600c0c5b3000000060004407800c9
:107fb80067ec070004c3b300844f5000faff3a008f
:107fc800ddff3700881f7800244a80004522de0044
:107fd800614262000044eb00e14f520006003200ab
:107fe80008003700a893200018447800e04f540098
:107ff8000100320044a9a800084078004f04780026
:10800800000006003ac9bf00c4ff0700c4c5b3009a
:10801800844f5000f8ff3a00f2ff3700881f7800bd
:10802800804278008143780004047800a6932000f9
:108038001643780021c5b300854f53002b003a0042
:108048002d00370014027800e00f520003003200c0
:10805800844a900082cf5200faff3a00f453880015
:1080680031c5b3007594200095427800e4cf5200e2
:108078001e003a00a594200095427800e0cf5200f7
:108088001a003a005029ef00784a8800e44090002e
:108098000140780052e9b7000340780053e9b7007f
:1080a8008783fb00674a88000240780054e9b700dc
:1080b8000540780046e9b7000382fb000500200070
:1080c8000801780006407800eaee07008040780052
:1080d800e0cf500003003a0010c0b3004ae9b700ef
:1080e800020037000140780046e9b70001407800f7
:1080f8004f04780000000600e4538000f453880021
:10810800d1ff3700a493200014427800804f52001a
:108118001000320024c5b300844878000049eb0001
:1081280010c0b300000006006494200014427800d8
:1081380084487800049520001442780004497800a7
:108148004ac9bf000080fb000000e9004f00de00c4
:10815800000006007494200014427800e04f52009a
:10816800f1ff3a00ebff3700a49320001442780097
:1081780025c5b300804f52000d003a000e003700ad
:1081880095027800e08f520003003200054b900002
:10819800814f5300faff3a00f5538800e5409000fc
:1081a800044078006ced07004a69ef008042eb005c
:1081b8000540780000000600e5538000f55388006c
:1081c800f0ff37000042780020c5b300a5932000d7
:1081d8009542780084cf520009003a000900370020
:1081e800e0c0b3004469b7004429a80040c0b30008
:1081f80048e9b7000040eb00fafe07000040eb003a
:10820800000006007494200014427800e14f5200e8
:10821800f3ff3e0080c5b300000006000000060022
:10822800889fbe008043780083427800040378006a
:10823800a99320009944780023c5b30087cf540040
:108248003b003a003d00370014027800e00f52006e
:1082580003003200844b900082cf5300faff3a00ab
:10826800f453880033c5b30077942000974378000f
:10827800e4cf53002e003a00689520001844780097
:10828800e04f54002a003a005c29ef00d64a8800e3
:10829800f4439000074078005ee9b7000540780095
:1082a8005fe9b7008181fb000390a000c34a880002
:1082b8000240780060e9b7000840780046e9b70056
:1082c800e0cf53000c003a00b49320001442780029
:1082d800841f78008582fb000282fb0092c0b300f5
:1082e80011c2b30009407800f5f307008041780017
:1082f8008f87e900070037000582fb000500200092
:10830800060178008740780009407800b7ee07003a
:1083180080417800e0cf510003003a0010c0b3005c
:1083280056e9b700020037000340780046e9b70075
:10833800034078004f04be0000000600e4538000ac
:10834800f4538800c1ff3700a4932000144278003a
:10835800804f52001000320024c5b30084487800d2
:108368000049eb0010c0b300000006006494200030
:108378001442780084487800c4952000144278009c
:108388000449780056c9bf000080fb000000e900de
:108398004f00de00000006007494200014427800ac
:1083a800e04f5200f1ff3a00ebff37000200fa00fd
:1083b800889fbe00004478000840780081ff0700cd
:1083c800b0ff9f00e04f500010003a00e9c5b3002d
:1083d80053f0070008407800d0fe0700b0ff9f0068
:1083e800894f5000faff320066815700e580570038
:1083f80008407800d4ff07000042780070c5b30039
:10840800e04f5200010032003ff897004f04be00d1
:108418000080fa0000000600a493200014427800af
:1084280025c5b300804f52000d003a000e003700fa
:1084380095027800e08f520003003200054b90004f
:10844800814f5300faff3a00f5538800f540900039
:1084580004407800c0ec07005669ef008042eb004a
:108468000540780000000600e5538000f5538800b9
:10847800f0ff3700ea874700889fbe008a9fbe004a
:108488008c9fbe008e1f78000003780001077800db
:1084980082047800030678000404780088057800d0
:1084a8000bf0a7008b05ea008b05e900cf5dde0025
:1084b8000c02780004f0a7000402ea000402e900b4
:1084c8004f22de0004c275000482fb008505780097
:1084d8000bf0a7008b05ea008b05e900cf5dde00f5
:1084e8008b0572000040eb00ed02200032003200e4
:1084f800370037000dd9b900020078002a09b40006
:1085080000057800908f14002a003a007482570002
:10851800f68157000e0178008600780085bf9f001d
:10852800f6b79f000c0707008fba97007fb3970034
:10853800e04f50001f0032006a0a90004322dd001d
:10854800040078002c09b40000037800164e780067
:108558002a639000afeb9700874a43006549800083
:10856800e08f540003003a00048242001402900095
:108578000b003700e18f540007003a0004824200e4
:1085880024029000670242004322de00044c780077
:10859800094078000e00370004824200340290003f
:1085a800670242004322de00044c780010c0b3008a
:1085b800070037008b05e800c48f200014427800bc
:1085c8000482fb00848f5500caff39000040eb008d
:1085d8004f0778004f06be004f05be004f04be008f
:1085e800af00b10000000600ee874700889fbe007c
:1085f8008a9fbe008c9fbe008e1f7800d0b79f0058
:108608008103780002047800030678008404780067
:10861800890578000bf0a7008b05ea008b05e900b7
:10862800cf5dde000c02780004f0a7000402ea0027
:108638000402e9004f22de0004c275000482fb0038
:10864800860578000bf0a7008b05ea008b05e9008a
:10865800cf5dde008b0572000502780004f0a700ec
:108668000402ea000402e9004f22de008485750056
:108678000040eb00ed0220002e00200040003200f8
:10868800440037000b80fb000d81b9000200780020
:108698002a09b40000057800900f140037003a004a
:1086a800201290000e02620034003200705a9000ce
:1086b800e14f5200310032007a825700f8815700aa
:1086c80007017800dfb09700f5b79f0086bf9f00cd
:1086d800e7b79f00a0060700ffb297000fbb9700ff
:1086e800efb39700e04f5000240032006a0a900070
:1086f8004322dd00040078002c09b40080037800d0
:10870800174e7800fa5b9000074b78007a5b900070
:108718000683fb008feb970007b3b9002a6090002f
:10872800864a400065498000e00f540003003a0083
:1087380004824200140290000b003700e10f54003d
:1087480007003a00048242002402900067024200b7
:108758004322de00844c7800084078000d00370082
:108768000482420034029000670242004322de0085
:10877800844c780010c0b300060037008b45e80031
:10878800c48f20001442780084cf5500bdff390003
:108798000040eb004f0778004f06be004f05be00b3
:1087a8004f04be00ef00b10000000600889fbe0025
:1087b8008a9fbe008c1f780000067800810478002c
:1087c800e00f56005200320093029000e08f5200f2
:1087d800050032001c4078000083fb000042eb00db
:1087e800868f52004b003a000042eb00938f140032
:1087f80048003a00c34290008582fb000504e90066
:10880800e34390008783fb00534390000683fb00fb
:1088180006bbb90086034400860020001100090049
:108828008603d800000378008000eb0018002000c1
:10883800890f53003000360036003700432dde0024
:10884800e7846200d34390000783fb000603e90036
:10885800050343004333de000002eb00010037004c
:108868000b0378004822dd00ec457b008b85fb007c
:10887800048275008605e9008a0f5300f8ff3e0060
:10888800e08f5400010032000922de00efcf5300d0
:1088980014003e008784fb000943dd000603e9005d
:1088a8000602620073439000e04f53000d0032004f
:1088b80016002000e1cf5300020036000903e9004a
:1088c8000643dd00860343008703e90004036300d1
:1088d80002003a0007026200020037008783ea00bc
:1088e8000702720004197800534290000482fb00ca
:1088f800848242008100e800634290000482fb0009
:10890800848f5000cdff390014c0b3000100370038
:108918000c427800044078004f0678004f05be00ee
:108928004f04be0000000600d4c8bf0000000600c7
:108938000200fa00889fbe008a1f78000042780073
:108948008204780025072000858f5000140032002b
:1089580009003e00ec825200858f5000050132006c
:10896800eb824200858f500007003200e08f5000f4
:1089780000013200dc00370064072000848f5000bb
:10898800d9003e00fb003700a993200099447800e5
:1089980018c0b30084cf5400d4003a00d800370080
:1089a8003ac9bf000044eb00844f5000cf003a00a2
:1089b800de00370099007800814a880079429000eb
:1089c800e04f52007b003a00f4538000940290007c
:1089d800858f500077003a00144990000281fb000f
:1089e80084499000004a8000c8020700000478000b
:1089f800184a8800e00f5400090032003ac9bf0045
:108a0800e2fc070060c5b30046e9b70090c0b300b8
:108a180047e9b7006022b8000001eb005a003700b0
:108a28006022b80008017800912520003ac9bf00eb
:108a380061070700e04f5000020032004489a80097
:108a480018003700f4538000844a90008582fb00a8
:108a580094942000144278000482fb000402e90088
:108a6800848f52000f003a00244a80004422de001e
:108a7800614262000b003a003ac9bf00c3fc07001c
:108a880060c5b30046e9b70090c0b30047e9b70036
:108a98006022b80008017800112620003ac9bf00fa
:108aa80045070700004a800005e907004029ef0054
:108ab800f453800014047800f8538800e00f540041
:108ac8002500320098029000e08f52000b0032001f
:108ad80005007800c5bf9f006be80700004a8800c2
:108ae800cfba9700e00f500004003a0050c0b3001e
:108af80046e9b70094c0b30014003700084a900054
:108b0800b693200016437800861f780017c0b3007c
:108b1800064a80000482fb000320220062c0b300e2
:108b280011c8b3003ac9bf00e5f107008f87e90013
:108b380024c0b300e04f500004003200004a800017
:108b4800dfe807004029ef008a003700044078007a
:108b580047e9b70087003700244a80004422de0036
:108b6800614262000a003a003ac9bf0087fc070068
:108b780060c5b30046e9b70090c0b30047e9b70045
:108b88006022b8000801780011262000060037008e
:108b980040c0b30047e9b70064002000050020008a
:108ba80062932000f12520003ac9bf0002070700a0
:108bb800700037008040eb0012eb07006d003700b3
:108bc800a894200018447800e14f54001a003a0095
:108bd800e9409000249520001442780084cf50008a
:108be80015003a0079459000e04f55000800320022
:108bf800f14f55001f0032000a40780046e9b700df
:108c080040c0b30047e9b7004a69ef0037003700b2
:108c1800fcea070099047800894a88000a4078002d
:108c280046e9b70040c0b30047e9b7000a407800fa
:108c38004ae9b7002d00370018c0b300649520003a
:108c480014427800884f520028003a00e94090000a
:108c5800e49520001442780084cf500023003a00a5
:108c680079459000e04f55000f003200f14f550054
:108c780007003a00e3ea070040c0b30048e9b7003c
:108c88004429a8000040eb0056fc070017003700f5
:108c98000a40780046e9b70040c0b30047e9b7008a
:108ca8005669ef0011003700d6ea070099047800ea
:108cb800e94a88000a40780046e9b70040c0b30096
:108cc80047e9b7000a40780056e9b70007003700bf
:108cd8007940900046e9b7004429a9000040eb001c
:108ce80040fc0700230037000044eb0008407800f0
:108cf8004f0578004f04be000080fa00000006000f
:108d08001400200005002000a29320000126200066
:108d180009407800a8060700094078001bfc0700f6
:108d28003a69ef004769ef00f0ff370074942000bc
:108d3800144278000482fb00050020006202520001
:108d4800e0825a00e70f5200e08f5a00e6ff3e002b
:108d58000460010017ff3700e3ff370098ff370072
:108d6800e1ff3700e0ff3700d9ff3700deff3700ab
:108d78000000370018c0b300dcff370010c0b30094
:108d880000000600889fbe008a9fbe008c9fbe0020
:108d980000447800a49320001442780010c0b30067
:108da800884f5200970032000040eb00804f52007d
:108db80094003a0097003700090245009442900059
:108dc800e4cf520057003a0054429000e34f52005b
:108dd80002003200e04f520052003a000d40780085
:108de80045e9b700a0002000a7e70700e00f500002
:108df80084003200e4538000e00f520004003a007f
:108e0800e0538800f0538800040878000400370015
:108e1800f4538000000a7800f05388000008eb0043
:108e2800f453800089024500a5429000054a980045
:108e3800eac27c008582fb008584440089024500e3
:108e4800154390008c4f530036003a00554390006c
:108e5800e04f530033003200054b90004833dd00eb
:108e6800f54290008582fb00850273001502980088
:108e7800eac27c008582fb00898442008042eb00c4
:108e8800854378000543780010003700b042900011
:108e9800e3cf52000a003a00a0429000e0cf52000f
:108ea80004003d00e04f530005003a0005437800f8
:108eb80003003700e0cf530001003a0085437800f3
:108ec800eac27c000580fb0080844400090045005c
:108ed80090409000e5cf5000ecff32008582fb0007
:108ee80085845400e04f53000e003200084078009b
:108ef8003ae9b7006642980077429800890245002f
:108f0800d5439000c83bdd00454390000683fb0035
:108f18000683730026029800e5429000154a9800df
:108f28001bc0b3006ac27c000482fb008484440036
:108f3800aa4290008582fb003a4290004822dd0058
:108f480005027200848f54009bff3900e0cf550062
:108f58002b003200e8538000f85388001802900074
:108f6800e00f520009003200004a8000e00f500074
:108f780001003200d2e707001800900042e707001e
:108f8800004a8800e00f50001e003200084a900096
:108f9800b593200095427800851f780017c0b3006c
:108fa800064a8000980290000482fb0003202200f9
:108fb80062c0b30011c8b3003ac9bf00c0f00700cf
:108fc800804278008f87e900e0cf52000500320028
:108fd800004a8000bae707004029ef000040eb0094
:108fe8000800370020c0b30047e9b7000540780003
:108ff8004ae9b70056e9b70010c0b30001003700ce
:109008000b4078004f06be004f05be004f04be005f
:1090180000000600d453800044a9a900044b900026
:109028000683fb00944a9000c82add0086827200fd
:10903800b5498800a44a90008582fb00344a900014
:109048004822dd0005027200c4498800014078000a
:109058003be9b700ca5380004a40900049e9b7008d
:109068008004eb00894578001dc0b3001cc2b30022
:10907800afff37000042eb0004407800f2e8b70089
:1090880016c0b30006407800f3e8b7008002eb0092
:10909800054788001547880005407800f8e8b700bc
:1090a80004407800f9e8b700fae8b700fce8b70030
:1090b80006407800fde8b70055478800044078006e
:1090c80000e9b70002e9b7008547880001e9b70061
:1090d800d5e8b700d6e8b700d7e8b700d8e8b700b2
:1090e800d9e8b700dae8b7006033b8005648880016
:1090f80067488800364888004748880096488800ae
:10910800a7488800764888008748880022e9b70081
:1091180020e9b700f548880021e9b700d64888005b
:10912800e7488800b6488800c7488800254888006e
:10913800000006008002780020002000e08f520026
:109148008a00320014922000144278000482fb0046
:1091580016002000070020000402e9000300330085
:109168000603430087834b00fbff3700d000200035
:109178005248800063488000860f5100878f59004d
:109188007a003d0080002000a48d20001442780061
:10919800e04f520075003a00948d20001442780088
:1091a800e04f520071003a0090002000848d2000aa
:1091b80014427800e04f52006c003a00748d200091
:1091c80014427800e04f520068003a00a0002000e6
:1091d800648d200014427800e04f520063003a008a
:1091e800548d200014427800e04f52005f003a008e
:1091f800c68f2000164378000680fb00e40220009a
:109208000481b900020078002a09b400000278003d
:109218000643e80006407800fce8b7001503900014
:10922800a50390002612980037129800e203420026
:10923800409020000f000900b01b7800b68f200076
:109248001643780036629800568f2000164378003f
:10925800066a980017902000974378000740780026
:10926800f5e8b70006c35300166a9800768f200009
:1092780016437800266a9800f78f200097437800f5
:1092880007407800f7e8b70006c35300366a98002d
:10929800668f200016437800466a9800478f2000a2
:1092a8009743780007407800f6e8b70006c35300f4
:1092b800566a9800f04880004300dd002c09b4008d
:1092c80027922000974378008783fb00169220009e
:1092d800164378000683fb0006bbb90095027800a8
:1092e800c42ade00ef826200e98f52000d003200ce
:1092f800eb8f520003003200e88f520018003a004a
:109308001000370025002000050a7800e042900090
:10931800256298003002900006034200360098004b
:109328000e00370015002000050a7800c0439000a1
:109338002762980020029000060342002600980049
:1093480006003700000aeb00a04290002562980052
:109358001002900006034200160098000000050065
:1093680035002000050a78000000eb000000060028
:109378009042780063c262001a003200100378003d
:10938800e3026300e38f520001003a0044c0b300d7
:109398008482fb008502e800e0c27a00e0cf520038
:1093a80010003d000c0037000483fb004333dd0050
:1093b800062bdd00cfb3de0010019000a001900065
:1093c8000603710087837100160098002700980033
:1093d8000442e80001003700f50f2000e44f520076
:1093e800f1ff3a000000060000037800348f2000e7
:1093f800144278008442e80005407800f3e8b7009a
:109408002549800004407800e2c0b3000440bc0055
:10941800028142003619780026117800568f200004
:109428001643780066419800568f2000164378004e
:1094380017902000174313007641980001c9bf0018
:10944800f5e8b700e68f20001643780046499800f3
:109458000043eb0006407800fee8b7003649980064
:109468002648800026019800c78f2000974378007f
:1094780007499800fbc8bf0020499800fbc8bf00f7
:10948800e2c0b3000440bc0082824200b44a9800a3
:10949800258f2000954278000583fb0097498000be
:1094a800fbc8bf0080737b008542e8000540780058
:1094b800f2e8b70004407800fbe8b70000000600b7
:1094c800fbc8bf00e2c0b3000440bc000200780043
:1094d8002409b400004a9000c58f200015421200ec
:1094e80014489800f248ed00f2e8b7000080fb004d
:1094f8009449800064427800fbc8bf00fee8b700ca
:1095080004407800fbe8b700000006000600fa00f7
:10951800889fbe008a9fbe008c9fbe000004be00cc
:10952800020578008345780021002000e00f5400f0
:10953800ff023200e08f5400fd023200208d20002f
:10954800280009000018eb00cafe07000b4078004d
:10955800d4e8b7009a4688008802780009027800a3
:109568008000eb0015417800e2ef9f00e3436100c3
:109578007fb397006300630046c0b300e30f500059
:1095880001003200074378008683fb008783ea00e6
:1095980007024200ffb397004238de006300600014
:1095a800e10f500024003200e20f50003b0032006f
:1095b800e00f500059003a004439de006f016100a5
:1095c800cf91de0068015100e0815900e40f51009d
:1095d800e08f590051003e0002600100140037007e
:1095e8001300370002003700110037000900370068
:1095f800f368ec00f248ec00f2e8b700978f20001f
:1096080097437800874f500044003600f9e8b700c8
:1096180042003700278f2000974378000740e90071
:10962800f2e8b700e0cf5300390032003b003700c2
:10963800fc68ec0039003700c43bde00ef836300b0
:10964800ea8f530006003200eb8f53000c00320003
:10965800e88f530031003a00fd68ec002f00370016
:10966800f848ec00f8e8b700a78f20009743780087
:10967800874f500029003600fae8b7002700370066
:10968800f848ed00f8e8b700a78f20009743780066
:10969800874f500020003e00200037004439de008c
:1096a8006f016100cf91de00e90f5100e08f590092
:1096b8001a003e0002600100090037000a00370066
:1096c800090037000e0037000f0037000e00370082
:1096d8001200370006003700070037000600370081
:1096e8000269ec000d003700f028ec000b00370091
:1096f8000069ec0009003700ea28ec000700370091
:10970800e228ec0005003700e028ec0003003700f1
:10971800310020000100370041002000e00f520016
:10972800040032000683fb000603e800868242003c
:109738008cff370001057800e08f50007c023a006a
:1097480051002000248f200014427800e04f52007e
:1097580077023a00338f200093417800610020009f
:10976800e1cf510072023200c78f20009743780082
:1097780071002000e0cf53006d0232008647800060
:10978800610263008100200069023a0054478000aa
:10979800e10262009100200065023a00054780005e
:1097a80061816200a100200061023a000603d10035
:1097b80020902000104343000640780002e9b700db
:1097c8000402d100019020001142420004407800b8
:1097d80000e9b7008502d10011478000818242006c
:1097e800154788008783fb00e102200001beb9000d
:1097f80003407800e2c0b3000440bc008c03410081
:10980800d18f2000914078008180fb00c308dd00e3
:109818008183430006407800a2c0b3000440bc0026
:1098280082834300a68f2000164378000683fb003e
:109838004233dd00850243000482fb0004824200bb
:109848004222dd00968f2000164378000683fb0035
:10985800060242000402420084854300a0498000b9
:10986800e00f50000100320095e507000b0078007a
:1098780005e5070000027800a449880011002000cf
:10988800e00f52002a02320024498800f3c8bf00c2
:10989800e2c0b3000440bc00020242005449880000
:1098a800c28f2000124178000281fb00e5022000ef
:1098b8000591b9000201420062498800d48f200056
:1098c800144278000482fb004322dd0004024100b8
:1098d8008449880002c9bf00a2c0b3000440bc008c
:1098e80002024200744988000590200095427800e1
:1098f8008582fb00c32add00050242003449880046
:1099080015478000c32add000502420094498800fb
:10991800958f2000954278008582fb008582420061
:109928000502420044498800d2fd0700244980000e
:10993800000aeb00341278008042eb00354a9800a8
:10994800054a980065429800454a9800254a9800bb
:10995800154a9800754298008002eb00250298008d
:109968006449800035029800150298002502980085
:10997800050a780098407800e1ef9f0063c2600014
:109988007fb19700e30361004bc0b300e38f53003e
:1099980001003200844578000804e80008017800d6
:1099a8006022b8000043eb000d0037003240780019
:1099b8000080fb00010020008681fb00c319dd0048
:1099c8008301e90003003300000040008180480063
:1099d800fbff370000027200818272000643e80034
:1099e8008b4f5300f1ff39000b83fb000604440042
:1099f80084bf9f0095bf9f007fb397004230de0071
:109a080063006000e10f50001b003200e20f5000bd
:109a18008f003200e00f5000a9013a004433de0005
:109a28006f036300cfb3de0068035300e0835b007d
:109a3800e40f5300e08f5b00a1013e0006600100c7
:109a48000400370003003700060037000100370024
:109a58000700370072805700b6fd070080007800c5
:109a680095013700708057005ffe070094013700aa
:109a780093fe0700920137004433de006f03630052
:109a8800cfb3de00eb0f5300e08f5b008c013e008c
:109a9800066001000b0037000c0037001200370089
:109aa800180037001e0037002400370084013700f3
:109ab80025003700290037004b0037004d003700dc
:109ac80059003700244888007d013700728057000c
:109ad80027fe07000fba97009fba970034488800fe
:109ae80045488800760137007280570020fe07003d
:109af8000fb897009fb897005048880061488800c1
:109b08006f0137007280570019fe07000fba9700df
:109b18009fba970074488800854888006801370014
:109b28007280570012fe07000fb897009fb8970081
:109b380090488800a148880061013700b44888002f
:109b4800c54888005e0137000440780021e9b70065
:109b5800e04f52007c01320059013700e00f5200fb
:109b6800e08f5a007a013200d78f2000974378009f
:109b7800604980000043eb00010037000643e8001d
:109b8800874f5300070031008680fb00c308dd00c3
:109b98006081780003002000840f5100858f5900f0
:109ba800f6ff3a00874f53000a003a008683fb000d
:109bb800c33bdd00870340000640e800fde8b7002e
:109bc800840b78008400200094039800a403980074
:109bd800b40398000ff0970020e9b7000683fb0054
:109be800f6488800360137000440780022e9b700bb
:109bf80033013700848f2000144278000480fb0072
:109c08004500dd002809b400419020000f0009003c
:109c1800311878000002b1000442e80004407800de
:109c2800f8e8b70026013700f848ed00f8e8b70073
:109c38000080fb004500dd00444980004190200081
:109c4800000142000f000900b21878001c0137001b
:109c58004430de006f006000cf80de00e90f500066
:109c6800e08f580016013e0000600100090037002f
:109c7800230037005a003700940037009d00370052
:109c8800b40037000e013700cc003700d800370089
:109c9800ef00370014902000144278000440780048
:109ca800a2c0b3000440bc00020078003009b40030
:109cb800000378000442e8000440780001e9b70096
:109cc800004beb00ffb0970063826000e30f520087
:109cd80006003a001fb99700120398000fba9700c0
:109ce800f40fb20024039800f500370024488000e0
:109cf800140398008fba970025039800f0003700e6
:109d0800968d200016437800e04f5300270032005c
:109d1800149020001442780004407800a2c0b300d8
:109d28000440bc00020078003009b4000003780049
:109d38000442e8000440780001e9b70014c0b30009
:109d4800044b7800ffb0970063826000e30f520075
:109d580006003a001fb99700120398000fba97003f
:109d6800f40fb20034039800040037002448800040
:109d7800140398008fba9700350398009602900054
:109d88002101200024478000848f520001003a00fe
:109d98008a0078006447800044039800b602900067
:109da800850f52003900310037003700e38f530028
:109db80004003a0025478800f40fb2007447880071
:109dc800040037000409f800e408f9000fbb970005
:109dd8007647880010c0b300dae8b700b80037004b
:109de800a68d200016437800e04f53002a00320069
:109df800149020001442780004407800a2c0b300f8
:109e08000440bc00020078003009b4000003780068
:109e18000442e8000440780001e9b70014c0b30028
:109e2800044b7800ffb0970063826000e30f520094
:109e380006003a001fb99700120398000fba97005e
:109e4800f40fb2004403980004003700244880004f
:109e5800140398008fba9700450398009602900063
:109e68002101200024478000848f520001003a001d
:109e78008a0078007447800034039800c602900076
:109e8800848f52000100310031012000d968ef00b1
:109e9800da68ef0088003700e38f530004003a00c7
:109ea80025478800f40fb200644788000400370093
:109eb8000409f800e408f9000fbb9700664788001a
:109ec80010c0b300d9e8b7007d003700448f2000e8
:109ed800144278000480fb004300dd002609b4002a
:109ee800800278000442e80004407800f4e8b700f3
:109ef8003b003700568d200016437800e04f530092
:109f080010003200448f2000144278000480fb00c7
:109f18004300dd002609b400800278000442e8000e
:109f280004407800f4e8b70014c0b300844a78000d
:109f38008fb89700a1029800e2468000b20298000c
:109f480017003700f446880010c0b300d6e8b70001
:109f58005b003700668d200016437800e04f530001
:109f680012003200448f2000144278000480fb0065
:109f78004300dd002609b400800278000442e800ae
:109f880004407800f4e8b70014c0b300844a7800ad
:109f98008fb89700b1029800f2468000a20298009c
:109fa800d668ef00d568ef0045003700e446880022
:109fb80010c0b300d5e8b70041003700f48f200087
:109fc800144278000480fb004300dd002e09b40031
:109fd800800278000442e80004407800ffe8b700f7
:109fe800804aeb008fb89700910298003400370040
:109ff800768d200016437800e04f530010003200a1
:10a00800f48f2000144278000480fb004300dd0038
:10a018002e09b400800278000442e8000440780069
:10a02800ffe8b70014c0b300844a78008fb89700df
:10a03800a102980032478000b2029800170037004a
:10a048004447880010c0b300d8e8b7001c003700a8
:10a05800868d200016437800e04f5300120032002e
:10a06800f48f2000144278000480fb004300dd00d8
:10a078002e09b400800278000442e8000440780009
:10a08800ffe8b70014c0b300844a78008fb897007f
:10a09800b102980042478000a2029800d868ef00f9
:10a0a800d768ef00060037003447880010c0b300b7
:10a0b800d7e8b70002003700e08f50001c003a00d4
:10a0c8008b85fb008b85ea008b84440029fe3a00cf
:10a0d8006649800015c0b300100037000582fb00f8
:10a0e8004322dd000402430094039000e88f5300ec
:10a0f80001003a0019029800a4039000e88f530069
:10a1080001003a0029029800b4039000e88f530038
:10a1180001003a00390298008542e800d48f2000f7
:10a128001442780084cf5200ecff39008a0078008e
:10a13800010078004f06be004f05be004f04be0068
:10a148000080fa0000000600f1002000f8ff370048
:10a1580001012000f6ff3700889fbe008a9fbe00dd
:10a168008c9fbe008002780002037800e08f5100c7
:10a178005b0032000504780008f0a7000804ea0034
:10a188000804e9004f44de0055003a00056d9000d0
:10a198008003eb0019c0b3004e0037000a40780076
:10a1a800a2c0b3000440bc00020078003009b4002b
:10a1b8008006780012002000e08f50000600320070
:10a1c8001d0190000281680002f0a7000201ea0068
:10a1d8000201e9004f11de008045eb009dcf15001c
:10a1e80024003200bd0590008b0f53001900390080
:10a1f8004d0690008c0f530016003e008b0553004f
:10a2080087894500e00f5200100032000886fb00e5
:10a218000c06e800956d90008b85fb008b0f5600af
:10a2280009003a00cd0590008b0f530006003a0054
:10a238008565900087c55500e1cf550002003600be
:10a248000b4a780001003700094a7800e04f5100b6
:10a2580025003a00cd0590008b05e8003d019000ef
:10a268000280550000f0a7000000ea008083430048
:10a27800160037002d009000800f530012003a009e
:10a2880087097800e00f52000d0032008885fb0036
:10a298008b05e800156890000080fb00808f550052
:10a2a80006003a000560900007405000e14f50005a
:10a2b80002003600004a780001003700094a780099
:10a2c800e04f510008003a008703e8000a45e8001b
:10a2d8000844e80015689000804f5400afff39002b
:10a2e8000040eb000100370010c0b3004f06be006d
:10a2f8004f05be004f04be0000000600c902a800ba
:10a30800c8e2a800c9c2a800c9e2a800c8a2a8005b
:10a31800c062a800c082a800c882a800c922a800fc
:10a328006360a8009660a8008660a9000000270066
:10a33800ac20b7009660a80000000600c902a8007b
:10a34800c8e2a800c9c2a800c9e2a800c8a2a8001b
:10a35800c062a800c082a800c882a800c922a800bc
:10a3680000000600e14f500003003a00c902a900ae
:10a37800cd02a90000000600c902a80000000600de
:10a38800e14f500007003a00c8e2a900cce2a9005a
:10a39800c9c2a900cdc2a900c9e2a900cde2a9009d
:10a3a80000000600c8e2a800c9c2a800c9e2a800c7
:10a3b80000000600e14f500003003a00c8a2a900bf
:10a3c800cca2a90000000600c8a2a8000000060050
:10a3d800c902a90010c0b300e2ff0700c8e2a90043
:10a3e800c9c2a900c9e2a90010c0b300e4ff070070
:10a3f800c8a2a90010c0b300eeff0700c062a90000
:10a40800c462a800c082a900c482a800c882a900aa
:10a41800cc82a800c922a900cd22a800000006000d
:10a42800e14f500003003a00c922a900cd22a9003b
:10a4380000000600c922a80000000600e14f5000f5
:10a4480003003a00c082a900c482a90000000600e7
:10a45800c082a80000000600e14f500003003a0047
:10a46800c882a900cc82a90000000600c882a80002
:10a4780000000600e14f500003003a00c062a90046
:10a48800c462a90000000600c062a800000006001f
:10a49800889fbe008004780064a7200014427800da
:10a4a8000482fb00e5a6200065407a00f1ff070062
:10a4b80064a72000144278000482fb0025a720002e
:10a4c80065407a00ddff07000004eb000400370058
:10a4d8000014200001002000ae0307000804e80073
:10a4e800890f5400faff35004f04be000000060033
:10a4f800889fbe008004780074a72000144278006a
:10a508000482fb00e5a6200065407a00d2ff070020
:10a5180074a72000144278000482fb0025a72000bd
:10a5280065407a00beff07000004eb000400370016
:10a538000014200001002000960307000804e8002a
:10a54800890f5400faff35004f04be0000000600d2
:10a55800cfff070065a72000954278000042eb0076
:10a56800e2cf520001003e000542e80004407800b6
:10a5780076eab70000000600c5ff070065a72000bf
:10a588009542780034c0b300e0cf52000100320099
:10a598000542e9000440780076eab70000000600aa
:10a5a800d3ff070075a720009542780034c0b30098
:10a5b800e0cf5200010032000542e9000440780073
:10a5c80077eab70000000600c9ff070075a720005a
:10a5d800954278000042eb00e2cf520001003e00b5
:10a5e8000542e8000440780077eab700000006005a
:10a5f800881f7800000278000204780065092000ae
:10a60800850f520003003c00a5f62f00850f52006d
:10a6180001003d000502780065092000858f500083
:10a6280003003c00a5f62f00858f500001003d0077
:10a63800850078008402780005f0a7008502ea000a
:10a648000540780006e8b7008102780005f0a70009
:10a658008502ea000540780007e8b70015c0b30096
:10a66800e00f520001003c008042eb0005407800fa
:10a6780008e8b70014c0b300e08f500001003c00a8
:10a688000042eb000440780009e8b7001a003700e0
:10a69800e04f52000a003200848020001442780003
:10a6a800e04f52000300320008007800b2ff0700b4
:10a6b8000200370008007800a5ff07000668ed00d3
:10a6c8007480200014427800e04f52000a003200e3
:10a6d8009480200014427800e04f520003003200ba
:10a6e80008007800aeff0700020037000800780075
:10a6f800b5ff07000768ed00648020001442780069
:10a708007680200096427200e1ff3a004f047800fc
:10a718000000060061006000610260004723dd0060
:10a72800f5f72f0067168000878262008682720024
:10a73800651688004e22dd00f5ff2b0066168000a6
:10a748008682620004827200641688004f00dd0071
:10a75800f4ff2700671680000702620000007200fd
:10a768006016880000000600caa2ab00feff3a008f
:10a7780000000600caa2ab00feff3200000006007f
:10a7880002003700caa2ab0002003a00cb02ab00bd
:10a79800fcff3a000000060002003700caa2ab0026
:10a7a80002003a00cb02ab00fcff320000000600ba
:10a7b800f3ff0700f8ff3700a4062000848f50003d
:10a7c80007003c000402e900848f50000e003d00a1
:10a7d80064025200848f50000e003a000a003700cd
:10a7e800c4062000848f50000a003500640242002d
:10a7f800848f50000400340094252000848f50007a
:10a8080004003a000200370010c0b3000000060040
:10a8180072f237000040eb00000006000400fa0066
:10a82800e0bf9f00f1bf9f00950180007fba9700ad
:10a83800940188006fba97001483ba0086007800e4
:10a848001400ba00950188000080fa000000060094
:10a85800404e200001002000f0ff070074c3b30041
:10a86800804f520018003a00604e2000010020007e
:10a87800eaff0700d4c2b300804f520012003a002a
:10a88800804e200001002000e4ff070024c6b3002a
:10a89800804f52000c003a00a04e2000010020001a
:10a8a800deff070094c6b300804f520006003a004e
:10a8b800c04e200001002000d8ff070044c7b300a5
:10a8c800804f52000b003200008028003101200028
:10a8d800b002070020002000a30207000080280023
:10a8e80031012000ab020700200020009a02070077
:10a8f800f5ff370000000600881f7800400120009f
:10a9080053020700b8cab300804f54001c0032003d
:10a91800b10a200040012000650207004001200024
:10a928004b020700804f54000a003a001100200033
:10a93800a00020005e02070011002000e0012000b6
:10a948005b020700a10020008002200058020700d7
:10a958000b003700200020008302070000602a0057
:10a96800e10020008b020700200020007a02070087
:10a9780000602a00e100200086020700f5ff37008a
:10a988004f04780000000600a000200030020700f5
:10a99800cf80de00204b8800314b8800e20f50004a
:10a9a800e08f5800050036006429ef006629ef00a3
:10a9b8008000eb00a00020003d02070024002000da
:10a9c800444b88006a29ef0080022000200207001b
:10a9d800cf80de00804b8800914b88002003200048
:10a9e8001b020700cf80de00604b8800714b880097
:10a9f800e10f5000e08f5800030036008000eb00a4
:10aa0800200320002a02070020032000100207006c
:10aa1800cf80de00604b8800714b88000000060084
:10aa28002ca3ef0020002000560207002000200081
:10aa38004902070000402c00910020005502070041
:10aa4800200020004802070000402c009100200050
:10aa580050020700200020003f02070000402c00a1
:10aa6800910020004b020700200020003e02070052
:10aa7800c022a800c9a2a900cda2a90004fe2f00e7
:10aa880035358000050262009400b3003435880033
:10aa9800f40f2e0065368000050262000550200084
:10aaa80005027200643688002100070068c0a8000b
:10aab80068e0a80000802400811e2000b80107007b
:10aac80063ff07008cff0700afff070000002500a9
:10aad800310c20002f02070010002000010207009f
:10aae8006000b800d3e307004df1070003fe07003c
:10aaf800104b80002400070089e60700c7f507000f
:10ab08004ef10700fcff370010c0b300000006003c
:10ab1800040024003604800086026200e08f5200a0
:10ab2800fcff3200b011800087c0a90000000600b9
:10ab380024022000c41188000002eb008411880060
:10ab48003062a8009411880031e2a8003342a800be
:10ab580087c0a90000000600000024008600b60097
:10ab68000000ea004f00de00000006000000fb00c5
:10ab7800a011880000000000000000003302ab00b4
:10ab8800feff320000000600881f780000047800ed
:10ab980001003700f5ff070038407800e04f50000b
:10aba800fcff3a004f04780000000600881f780078
:10abb800004478000042eb0035c6b300854f5400ce
:10abc800070036000880fb00440620001100090039
:10abd8000480d8000043b000e4ff070014c0b300ad
:10abe8000884fb0045062000110009000584d800f0
:10abf80001447800e94f540002003e00e14f520042
:10ac080006003a000880fb00a4002000110009009b
:10ac18000480d8000043b000d4ff07000884fb007c
:10ac2800a4002000110009000484d80004c3b30064
:10ac380004c04000cdff07004f0478000000060064
:10ac4800889fbe008004780044cade006f0262005c
:10ac58004889290068407a00c4ff0700ef8464002f
:10ac680068c07c00c1ff07004f04be00000006005a
:10ac7800889fbe00800478004c4ade00488929007d
:10ac880068407a00b9ff0700484ade006f02620098
:10ac980068407a00b5ff0700444ade006f02620090
:10aca80068407a00b1ff0700ef84640068c07c0048
:10acb800aeff07004f04be0000000600889fbe00dc
:10acc8008a9fbe000005be004c0ade000500200079
:10acd8004889290068407a00a4ff0700485ade0026
:10ace80005002000f90020000482640068407a0012
:10acf8009eff0700445ade0005002000048264001d
:10ad080068407a0099ff07000b82640068407a0067
:10ad180096ff0700445bdd004c52de00040273001e
:10ad2800cc5ade000482640068407a008fff070076
:10ad3800485bdd004852de0004027300c85ade009a
:10ad48000482640068407a0088ff07004c5bdd00dd
:10ad58004452de0004027300c45ade000482640018
:10ad680068407a0081ff07000a85640068407d001a
:10ad78007eff07004f05be004f04be00000006001e
:10ad88000042eb0065c6b300854f500015003c003b
:10ad9800e6c25200854f50000200340094cab30046
:10ada8000f00370065c4b300854f50000d003c000c
:10adb800e6c25200854f50000200340094ccb30024
:10adc8000700370095c3b300854f500005003c00cd
:10add800eac25200854f50000200340004cdb3008f
:10ade8000442400004407800000006006f40600004
:10adf800e94f5000020034007043b0000000060024
:10ae08000043b000000006003222ab00010032000f
:10ae18003222a9000000060000037800a4c0b30095
:10ae28000040eb0045972000a2c0b3000440bc00de
:10ae3800e5037900868f530002003a000281420040
:10ae48000009eb000040e8000442e900f6ff3a0080
:10ae580000000600000278000203be00d8c9bf0047
:10ae680016003200a5c0b3000040eb00a2c0b3003a
:10ae78000440bc0041972000e1017900e08f5100b7
:10ae88000a003a00843079000182e8000202420098
:10ae9800068abe0066824000020142000009eb00fb
:10aea8003211780010c0b300000006000040e8002e
:10aeb8008542e900edff3a000540780000000600f1
:10aec800e00f500003003200e10f500016003a0076
:10aed800120037004497200031000900001aeb00e7
:10aee800440580000400a0000410a1000420a10073
:10aef800440588008500a9005008880004d0270070
:10af08007408880004002a00940888009500a800a6
:10af180010c0b300d8e9b700000006009500a900ea
:10af2800d869ef00000006000040eb0000000600b2
:10af38003600f800809fbe00829fbe00849fbe003e
:10af4800869fbe00889fbe008a9fbe008c1f780027
:10af58003400f80000002000a0018800a9c0b30058
:10af68008045eb0048972000660544000b407800b8
:10af7800a2c0b3000440bc0068027900e00f520090
:10af880010003200e6024100850244001000200053
:10af98000100200035034000a58348000206450053
:10afa800068ebe000281e80002014400b20f530081
:10afb800a28f5b0003003a0004000100000eeb00c2
:10afc8003c1678008b45e8008944e900e7ff3a0021
:10afd8008500a9003400f9004f0678004f05be002f
:10afe8004f04be004f03be004f02be004f01be001b
:0caff8004f00be003600f90000400600cb
:020000040000fa
:10b00400740900006600000000000000da09000076
:10b014001a00000002000000c6469c004400000024
:10b024000000000000030100020000000002000014
:10b03400030000000000000002000000780a000085
:10b0440004000000020000000000000000000000f6
:10b05400100a00005e00000000000000000a00006a
:10b064001000000000000000360900002c00000061
:10b07400000000007c0a0000040000000000000042
:10b08400d20800006400000002000000000000007c
:10b0940000000000000000000000000000000000ac
:10b0a400000000000000000000000000000000009c
:10b0b400000000000000000000000000000000008c
:10b0c400000000000000000000000000000000007c
:10b0d400000000000000000000000000000000006c
:10b0e400000000000000000000000000000000005c
:10b0f400000000000000000000000000000000004c
:10b10400000000000000000000000000000000003b
:10b1140000000000f40900000c0000000200000020
:10b12400000000000000000000000000000000001b
:10b1340000080000d20000000000000062090000c6
:10b144001200000002000000489801000000000006
:10b15400010000000000000000000a0000000000e0
:10b16400800a000002000000000000006e0a0000d7
:10b174000a000000020000000000010001000100bc
:10b184000100030003000000820a00001000000018
:10b1940000000000920a000002000000000000000d
:04b1a40000000000a7
:020000040000fa
:10b1a80002502300c300200098de07008000e90059
:10b1b800f0272d0084de070044de07000403280082
:10b1c800240888000021ef003406200005088000cc
:10b1d800848f5200fdff360000000600889fbe00e5
:10b1e8008a9fbe000005780047d4de006e04640024
:10b1f800080ab300890c20000b0028007bde07003a
:10b2080032de0700084078005ade07002fde07000c
:10b21800c510800005826500e00f5200050032006d
:10b2280076de070029de07008904e900f3ff3a000b
:10b238000084eb000a4078004ede070023de07009a
:10b24800080078004f05be004f04be00000006004d
:10b25800889fbe00e1ff07000004780067de070052
:10b268001ade070061de070018de07000840e80064
:10b2780040de070015de070031de07000084fb0012
:10b288000dde070011de07002dde07008044780080
:10b2980048de07000dde070058de07000bde07005a
:10b2a8004848dd00080070004f04be00000006009a
:10b2b800881f780001047800c8ff0700084078005c
:10b2c8002cde070001de070048c0de0029de07008b
:10b2d800fedd070049de0700fcdd07004f047800ab
:10b2e80000000600881f78000004780044a7a80022
:10b2f800e00f540006003a0020002000210007005b
:10b30800200020001400070008007800ecfe070069
:10b318004f047800000006003600f800809fbe0049
:10b32800829fbe00849fbe00869fbe003400f80046
:10b3380000002000a00188009aea07003400f90004
:10b348004f03be004f02be004f01be004f00be00bb
:10b358003600f90000400600e20f500001003a00f4
:10b36800c202a80000000600e20f500001003a00e7
:10b37800c202a90000000600000006000040eb0021
:10b3880000000600e20f500001003a00c002a900c8
:04b3980000000600ab
:020000040000fa
:10b39c00f03fb1000180b10006003500ee0309005a
:10b3ac0000000000403fb1000180b100fbff3d00f8
:10b3bc001000b000203fb0000200350000800900f2
:08b3cc00000000000000060073
:020000040000fa
:08b3d4000040da000000fe0059
:020000040000fa
:020000040001f9
:0457f00033ff000083
:020000040000fa
:020000040001f9
:0457f400c0f40000fd
:020000040000fa
:020000040001f9
:0457f8008f09000015
:020000040000fa
:020000040001f9
:0457fc00601f00002a
:00000001FF
